Archive member included to satisfy reference by file (symbol)

/opt/ti/ccsv7/tools/compiler/gcc-arm-none-eabi-6-2017-q1-update/bin/../lib/gcc/arm-none-eabi/6.3.1/../../../../arm-none-eabi/lib/thumb/v7e-m/fpv4-sp/hard/libc_nano.a(lib_a-exit.o)
                              /opt/ti/ccsv7/tools/compiler/gcc-arm-none-eabi-6-2017-q1-update/bin/../lib/gcc/arm-none-eabi/6.3.1/../../../../arm-none-eabi/lib/thumb/v7e-m/fpv4-sp/hard/crt0.o (exit)
/opt/ti/ccsv7/tools/compiler/gcc-arm-none-eabi-6-2017-q1-update/bin/../lib/gcc/arm-none-eabi/6.3.1/../../../../arm-none-eabi/lib/thumb/v7e-m/fpv4-sp/hard/libc_nano.a(lib_a-impure.o)
                              /opt/ti/ccsv7/tools/compiler/gcc-arm-none-eabi-6-2017-q1-update/bin/../lib/gcc/arm-none-eabi/6.3.1/../../../../arm-none-eabi/lib/thumb/v7e-m/fpv4-sp/hard/libc_nano.a(lib_a-exit.o) (_global_impure_ptr)
/opt/ti/ccsv7/tools/compiler/gcc-arm-none-eabi-6-2017-q1-update/bin/../lib/gcc/arm-none-eabi/6.3.1/../../../../arm-none-eabi/lib/thumb/v7e-m/fpv4-sp/hard/libc_nano.a(lib_a-init.o)
                              /opt/ti/ccsv7/tools/compiler/gcc-arm-none-eabi-6-2017-q1-update/bin/../lib/gcc/arm-none-eabi/6.3.1/../../../../arm-none-eabi/lib/thumb/v7e-m/fpv4-sp/hard/crt0.o (__libc_init_array)
/opt/ti/ccsv7/tools/compiler/gcc-arm-none-eabi-6-2017-q1-update/bin/../lib/gcc/arm-none-eabi/6.3.1/../../../../arm-none-eabi/lib/thumb/v7e-m/fpv4-sp/hard/libc_nano.a(lib_a-memset.o)
                              /opt/ti/ccsv7/tools/compiler/gcc-arm-none-eabi-6-2017-q1-update/bin/../lib/gcc/arm-none-eabi/6.3.1/../../../../arm-none-eabi/lib/thumb/v7e-m/fpv4-sp/hard/crt0.o (memset)
/opt/ti/ccsv7/tools/compiler/gcc-arm-none-eabi-6-2017-q1-update/bin/../lib/gcc/arm-none-eabi/6.3.1/../../../../arm-none-eabi/lib/thumb/v7e-m/fpv4-sp/hard/libnosys.a(_exit.o)
                              /opt/ti/ccsv7/tools/compiler/gcc-arm-none-eabi-6-2017-q1-update/bin/../lib/gcc/arm-none-eabi/6.3.1/../../../../arm-none-eabi/lib/thumb/v7e-m/fpv4-sp/hard/libc_nano.a(lib_a-exit.o) (_exit)
/home/student/git/workspace_mct/YAHAL/libYAHAL_msp432.a(gpio_msp432.cpp.o)
                              Debug/main.cpp.o (gpio_msp432::inst)
/home/student/git/workspace_mct/YAHAL/libYAHAL_msp432.a(timer_msp432.cpp.o)
                              Debug/main.cpp.o (timer_msp432::timer_msp432(Timer32_Type*))
/opt/ti/ccsv7/tools/compiler/gcc-arm-none-eabi-6-2017-q1-update/bin/../lib/gcc/arm-none-eabi/6.3.1/../../../../arm-none-eabi/lib/thumb/v7e-m/fpv4-sp/hard/libstdc++_nano.a(class_type_info.o)
                              /home/student/git/workspace_mct/YAHAL/libYAHAL_msp432.a(gpio_msp432.cpp.o) (vtable for __cxxabiv1::__class_type_info)
/opt/ti/ccsv7/tools/compiler/gcc-arm-none-eabi-6-2017-q1-update/bin/../lib/gcc/arm-none-eabi/6.3.1/../../../../arm-none-eabi/lib/thumb/v7e-m/fpv4-sp/hard/libstdc++_nano.a(atexit_arm.o)
                              /home/student/git/workspace_mct/YAHAL/libYAHAL_msp432.a(gpio_msp432.cpp.o) (__aeabi_atexit)
/opt/ti/ccsv7/tools/compiler/gcc-arm-none-eabi-6-2017-q1-update/bin/../lib/gcc/arm-none-eabi/6.3.1/../../../../arm-none-eabi/lib/thumb/v7e-m/fpv4-sp/hard/libstdc++_nano.a(si_class_type_info.o)
                              /home/student/git/workspace_mct/YAHAL/libYAHAL_msp432.a(gpio_msp432.cpp.o) (vtable for __cxxabiv1::__si_class_type_info)
/opt/ti/ccsv7/tools/compiler/gcc-arm-none-eabi-6-2017-q1-update/bin/../lib/gcc/arm-none-eabi/6.3.1/../../../../arm-none-eabi/lib/thumb/v7e-m/fpv4-sp/hard/libstdc++_nano.a(del_ops.o)
                              /opt/ti/ccsv7/tools/compiler/gcc-arm-none-eabi-6-2017-q1-update/bin/../lib/gcc/arm-none-eabi/6.3.1/../../../../arm-none-eabi/lib/thumb/v7e-m/fpv4-sp/hard/libstdc++_nano.a(class_type_info.o) (operator delete(void*, unsigned int))
/opt/ti/ccsv7/tools/compiler/gcc-arm-none-eabi-6-2017-q1-update/bin/../lib/gcc/arm-none-eabi/6.3.1/../../../../arm-none-eabi/lib/thumb/v7e-m/fpv4-sp/hard/libstdc++_nano.a(del_op.o)
                              /home/student/git/workspace_mct/YAHAL/libYAHAL_msp432.a(gpio_msp432.cpp.o) (operator delete(void*))
/opt/ti/ccsv7/tools/compiler/gcc-arm-none-eabi-6-2017-q1-update/bin/../lib/gcc/arm-none-eabi/6.3.1/../../../../arm-none-eabi/lib/thumb/v7e-m/fpv4-sp/hard/libstdc++_nano.a(pure.o)
                              /home/student/git/workspace_mct/YAHAL/libYAHAL_msp432.a(gpio_msp432.cpp.o) (__cxa_pure_virtual)
/opt/ti/ccsv7/tools/compiler/gcc-arm-none-eabi-6-2017-q1-update/bin/../lib/gcc/arm-none-eabi/6.3.1/../../../../arm-none-eabi/lib/thumb/v7e-m/fpv4-sp/hard/libstdc++_nano.a(tinfo.o)
                              /opt/ti/ccsv7/tools/compiler/gcc-arm-none-eabi-6-2017-q1-update/bin/../lib/gcc/arm-none-eabi/6.3.1/../../../../arm-none-eabi/lib/thumb/v7e-m/fpv4-sp/hard/libstdc++_nano.a(class_type_info.o) (std::type_info::~type_info())
/opt/ti/ccsv7/tools/compiler/gcc-arm-none-eabi-6-2017-q1-update/bin/../lib/gcc/arm-none-eabi/6.3.1/../../../../arm-none-eabi/lib/thumb/v7e-m/fpv4-sp/hard/libstdc++_nano.a(eh_terminate.o)
                              /opt/ti/ccsv7/tools/compiler/gcc-arm-none-eabi-6-2017-q1-update/bin/../lib/gcc/arm-none-eabi/6.3.1/../../../../arm-none-eabi/lib/thumb/v7e-m/fpv4-sp/hard/libstdc++_nano.a(pure.o) (std::terminate())
/opt/ti/ccsv7/tools/compiler/gcc-arm-none-eabi-6-2017-q1-update/bin/../lib/gcc/arm-none-eabi/6.3.1/../../../../arm-none-eabi/lib/thumb/v7e-m/fpv4-sp/hard/libstdc++_nano.a(eh_term_handler.o)
                              /opt/ti/ccsv7/tools/compiler/gcc-arm-none-eabi-6-2017-q1-update/bin/../lib/gcc/arm-none-eabi/6.3.1/../../../../arm-none-eabi/lib/thumb/v7e-m/fpv4-sp/hard/libstdc++_nano.a(eh_terminate.o) (__cxxabiv1::__terminate_handler)
/opt/ti/ccsv7/tools/compiler/gcc-arm-none-eabi-6-2017-q1-update/bin/../lib/gcc/arm-none-eabi/6.3.1/../../../../arm-none-eabi/lib/thumb/v7e-m/fpv4-sp/hard/libstdc++_nano.a(eh_unex_handler.o)
                              /opt/ti/ccsv7/tools/compiler/gcc-arm-none-eabi-6-2017-q1-update/bin/../lib/gcc/arm-none-eabi/6.3.1/../../../../arm-none-eabi/lib/thumb/v7e-m/fpv4-sp/hard/libstdc++_nano.a(eh_terminate.o) (__cxxabiv1::__unexpected_handler)
/opt/ti/ccsv7/tools/compiler/gcc-arm-none-eabi-6-2017-q1-update/bin/../lib/gcc/arm-none-eabi/6.3.1/../../../../arm-none-eabi/lib/thumb/v7e-m/fpv4-sp/hard/libc_nano.a(lib_a-abort.o)
                              /opt/ti/ccsv7/tools/compiler/gcc-arm-none-eabi-6-2017-q1-update/bin/../lib/gcc/arm-none-eabi/6.3.1/../../../../arm-none-eabi/lib/thumb/v7e-m/fpv4-sp/hard/libstdc++_nano.a(eh_terminate.o) (abort)
/opt/ti/ccsv7/tools/compiler/gcc-arm-none-eabi-6-2017-q1-update/bin/../lib/gcc/arm-none-eabi/6.3.1/../../../../arm-none-eabi/lib/thumb/v7e-m/fpv4-sp/hard/libc_nano.a(lib_a-cxa_atexit.o)
                              /opt/ti/ccsv7/tools/compiler/gcc-arm-none-eabi-6-2017-q1-update/bin/../lib/gcc/arm-none-eabi/6.3.1/../../../../arm-none-eabi/lib/thumb/v7e-m/fpv4-sp/hard/libstdc++_nano.a(atexit_arm.o) (__cxa_atexit)
/opt/ti/ccsv7/tools/compiler/gcc-arm-none-eabi-6-2017-q1-update/bin/../lib/gcc/arm-none-eabi/6.3.1/../../../../arm-none-eabi/lib/thumb/v7e-m/fpv4-sp/hard/libc_nano.a(lib_a-malloc.o)
                              /opt/ti/ccsv7/tools/compiler/gcc-arm-none-eabi-6-2017-q1-update/bin/../lib/gcc/arm-none-eabi/6.3.1/../../../../arm-none-eabi/lib/thumb/v7e-m/fpv4-sp/hard/libstdc++_nano.a(del_op.o) (free)
/opt/ti/ccsv7/tools/compiler/gcc-arm-none-eabi-6-2017-q1-update/bin/../lib/gcc/arm-none-eabi/6.3.1/../../../../arm-none-eabi/lib/thumb/v7e-m/fpv4-sp/hard/libc_nano.a(lib_a-nano-freer.o)
                              /opt/ti/ccsv7/tools/compiler/gcc-arm-none-eabi-6-2017-q1-update/bin/../lib/gcc/arm-none-eabi/6.3.1/../../../../arm-none-eabi/lib/thumb/v7e-m/fpv4-sp/hard/libc_nano.a(lib_a-malloc.o) (_free_r)
/opt/ti/ccsv7/tools/compiler/gcc-arm-none-eabi-6-2017-q1-update/bin/../lib/gcc/arm-none-eabi/6.3.1/../../../../arm-none-eabi/lib/thumb/v7e-m/fpv4-sp/hard/libc_nano.a(lib_a-nano-mallocr.o)
                              /opt/ti/ccsv7/tools/compiler/gcc-arm-none-eabi-6-2017-q1-update/bin/../lib/gcc/arm-none-eabi/6.3.1/../../../../arm-none-eabi/lib/thumb/v7e-m/fpv4-sp/hard/libc_nano.a(lib_a-malloc.o) (_malloc_r)
/opt/ti/ccsv7/tools/compiler/gcc-arm-none-eabi-6-2017-q1-update/bin/../lib/gcc/arm-none-eabi/6.3.1/../../../../arm-none-eabi/lib/thumb/v7e-m/fpv4-sp/hard/libc_nano.a(lib_a-on_exit_args.o)
                              /opt/ti/ccsv7/tools/compiler/gcc-arm-none-eabi-6-2017-q1-update/bin/../lib/gcc/arm-none-eabi/6.3.1/../../../../arm-none-eabi/lib/thumb/v7e-m/fpv4-sp/hard/libc_nano.a(lib_a-cxa_atexit.o) (__on_exit_args)
/opt/ti/ccsv7/tools/compiler/gcc-arm-none-eabi-6-2017-q1-update/bin/../lib/gcc/arm-none-eabi/6.3.1/../../../../arm-none-eabi/lib/thumb/v7e-m/fpv4-sp/hard/libc_nano.a(lib_a-sbrkr.o)
                              /opt/ti/ccsv7/tools/compiler/gcc-arm-none-eabi-6-2017-q1-update/bin/../lib/gcc/arm-none-eabi/6.3.1/../../../../arm-none-eabi/lib/thumb/v7e-m/fpv4-sp/hard/libc_nano.a(lib_a-nano-mallocr.o) (_sbrk_r)
/opt/ti/ccsv7/tools/compiler/gcc-arm-none-eabi-6-2017-q1-update/bin/../lib/gcc/arm-none-eabi/6.3.1/../../../../arm-none-eabi/lib/thumb/v7e-m/fpv4-sp/hard/libc_nano.a(lib_a-signal.o)
                              /opt/ti/ccsv7/tools/compiler/gcc-arm-none-eabi-6-2017-q1-update/bin/../lib/gcc/arm-none-eabi/6.3.1/../../../../arm-none-eabi/lib/thumb/v7e-m/fpv4-sp/hard/libc_nano.a(lib_a-abort.o) (raise)
/opt/ti/ccsv7/tools/compiler/gcc-arm-none-eabi-6-2017-q1-update/bin/../lib/gcc/arm-none-eabi/6.3.1/../../../../arm-none-eabi/lib/thumb/v7e-m/fpv4-sp/hard/libc_nano.a(lib_a-signalr.o)
                              /opt/ti/ccsv7/tools/compiler/gcc-arm-none-eabi-6-2017-q1-update/bin/../lib/gcc/arm-none-eabi/6.3.1/../../../../arm-none-eabi/lib/thumb/v7e-m/fpv4-sp/hard/libc_nano.a(lib_a-signal.o) (_kill_r)
/opt/ti/ccsv7/tools/compiler/gcc-arm-none-eabi-6-2017-q1-update/bin/../lib/gcc/arm-none-eabi/6.3.1/../../../../arm-none-eabi/lib/thumb/v7e-m/fpv4-sp/hard/libc_nano.a(lib_a-strcmp.o)
                              /opt/ti/ccsv7/tools/compiler/gcc-arm-none-eabi-6-2017-q1-update/bin/../lib/gcc/arm-none-eabi/6.3.1/../../../../arm-none-eabi/lib/thumb/v7e-m/fpv4-sp/hard/libstdc++_nano.a(tinfo.o) (strcmp)
/opt/ti/ccsv7/tools/compiler/gcc-arm-none-eabi-6-2017-q1-update/bin/../lib/gcc/arm-none-eabi/6.3.1/../../../../arm-none-eabi/lib/thumb/v7e-m/fpv4-sp/hard/libc_nano.a(lib_a-mlock.o)
                              /opt/ti/ccsv7/tools/compiler/gcc-arm-none-eabi-6-2017-q1-update/bin/../lib/gcc/arm-none-eabi/6.3.1/../../../../arm-none-eabi/lib/thumb/v7e-m/fpv4-sp/hard/libc_nano.a(lib_a-nano-freer.o) (__malloc_lock)
/opt/ti/ccsv7/tools/compiler/gcc-arm-none-eabi-6-2017-q1-update/bin/../lib/gcc/arm-none-eabi/6.3.1/../../../../arm-none-eabi/lib/thumb/v7e-m/fpv4-sp/hard/libc_nano.a(lib_a-reent.o)
                              /opt/ti/ccsv7/tools/compiler/gcc-arm-none-eabi-6-2017-q1-update/bin/../lib/gcc/arm-none-eabi/6.3.1/../../../../arm-none-eabi/lib/thumb/v7e-m/fpv4-sp/hard/libc_nano.a(lib_a-sbrkr.o) (errno)
/opt/ti/ccsv7/tools/compiler/gcc-arm-none-eabi-6-2017-q1-update/bin/../lib/gcc/arm-none-eabi/6.3.1/../../../../arm-none-eabi/lib/thumb/v7e-m/fpv4-sp/hard/libnosys.a(getpid.o)
                              /opt/ti/ccsv7/tools/compiler/gcc-arm-none-eabi-6-2017-q1-update/bin/../lib/gcc/arm-none-eabi/6.3.1/../../../../arm-none-eabi/lib/thumb/v7e-m/fpv4-sp/hard/libc_nano.a(lib_a-signalr.o) (_getpid)
/opt/ti/ccsv7/tools/compiler/gcc-arm-none-eabi-6-2017-q1-update/bin/../lib/gcc/arm-none-eabi/6.3.1/../../../../arm-none-eabi/lib/thumb/v7e-m/fpv4-sp/hard/libnosys.a(kill.o)
                              /opt/ti/ccsv7/tools/compiler/gcc-arm-none-eabi-6-2017-q1-update/bin/../lib/gcc/arm-none-eabi/6.3.1/../../../../arm-none-eabi/lib/thumb/v7e-m/fpv4-sp/hard/libc_nano.a(lib_a-signalr.o) (_kill)
/opt/ti/ccsv7/tools/compiler/gcc-arm-none-eabi-6-2017-q1-update/bin/../lib/gcc/arm-none-eabi/6.3.1/../../../../arm-none-eabi/lib/thumb/v7e-m/fpv4-sp/hard/libnosys.a(sbrk.o)
                              /opt/ti/ccsv7/tools/compiler/gcc-arm-none-eabi-6-2017-q1-update/bin/../lib/gcc/arm-none-eabi/6.3.1/../../../../arm-none-eabi/lib/thumb/v7e-m/fpv4-sp/hard/libc_nano.a(lib_a-sbrkr.o) (_sbrk)

Allocating common symbols
Common symbol       size              file

errno               0x4               /opt/ti/ccsv7/tools/compiler/gcc-arm-none-eabi-6-2017-q1-update/bin/../lib/gcc/arm-none-eabi/6.3.1/../../../../arm-none-eabi/lib/thumb/v7e-m/fpv4-sp/hard/libc_nano.a(lib_a-reent.o)

Discarded input sections

 .group         0x0000000000000000        0x8 Debug/main.cpp.o
 .group         0x0000000000000000        0x8 Debug/main.cpp.o
 .group         0x0000000000000000        0x8 Debug/main.cpp.o
 .group         0x0000000000000000        0x8 Debug/main.cpp.o
 .group         0x0000000000000000        0x8 Debug/main.cpp.o
 .group         0x0000000000000000        0xc /home/student/git/workspace_mct/YAHAL/libYAHAL_msp432.a(gpio_msp432.cpp.o)
 .group         0x0000000000000000        0xc /home/student/git/workspace_mct/YAHAL/libYAHAL_msp432.a(gpio_msp432.cpp.o)
 .group         0x0000000000000000        0x8 /home/student/git/workspace_mct/YAHAL/libYAHAL_msp432.a(gpio_msp432.cpp.o)
 .group         0x0000000000000000        0x8 /home/student/git/workspace_mct/YAHAL/libYAHAL_msp432.a(gpio_msp432.cpp.o)
 .group         0x0000000000000000        0x8 /home/student/git/workspace_mct/YAHAL/libYAHAL_msp432.a(gpio_msp432.cpp.o)
 .group         0x0000000000000000        0x8 /home/student/git/workspace_mct/YAHAL/libYAHAL_msp432.a(gpio_msp432.cpp.o)
 .group         0x0000000000000000        0x8 /home/student/git/workspace_mct/YAHAL/libYAHAL_msp432.a(gpio_msp432.cpp.o)
 .group         0x0000000000000000        0x8 /home/student/git/workspace_mct/YAHAL/libYAHAL_msp432.a(timer_msp432.cpp.o)
 .group         0x0000000000000000        0xc /home/student/git/workspace_mct/YAHAL/libYAHAL_msp432.a(timer_msp432.cpp.o)
 .group         0x0000000000000000        0x8 /home/student/git/workspace_mct/YAHAL/libYAHAL_msp432.a(timer_msp432.cpp.o)
 .group         0x0000000000000000        0x8 /home/student/git/workspace_mct/YAHAL/libYAHAL_msp432.a(timer_msp432.cpp.o)
 .group         0x0000000000000000        0x8 /home/student/git/workspace_mct/YAHAL/libYAHAL_msp432.a(timer_msp432.cpp.o)

Memory Configuration

Name             Origin             Length             Attributes
MAIN_FLASH       0x0000000000000000 0x0000000000040000 xr
INFO_FLASH       0x0000000000200000 0x0000000000004000 xr
SRAM_CODE        0x0000000001000000 0x0000000000010000 xrw
SRAM_DATA        0x0000000020000000 0x0000000000010000 rw
*default*        0x0000000000000000 0xffffffffffffffff

Linker script and memory map

LOAD /opt/ti/ccsv7/tools/compiler/gcc-arm-none-eabi-6-2017-q1-update/bin/../lib/gcc/arm-none-eabi/6.3.1/thumb/v7e-m/fpv4-sp/hard/crti.o
LOAD /opt/ti/ccsv7/tools/compiler/gcc-arm-none-eabi-6-2017-q1-update/bin/../lib/gcc/arm-none-eabi/6.3.1/thumb/v7e-m/fpv4-sp/hard/crtbegin.o
LOAD /opt/ti/ccsv7/tools/compiler/gcc-arm-none-eabi-6-2017-q1-update/bin/../lib/gcc/arm-none-eabi/6.3.1/../../../../arm-none-eabi/lib/thumb/v7e-m/fpv4-sp/hard/crt0.o
                0x0000000000000000                PROVIDE (_intvecs_base_address, DEFINED (_intvecs_base_address)?_intvecs_base_address:0x0)

.intvecs        0x0000000000000000       0xe4
 *(.intvecs)
 .intvecs       0x0000000000000000       0xe4 Debug/startup_msp432p401r_gcc.c.o
                0x0000000000000000                interruptVectors
                0x0000000000200000                PROVIDE (_mailbox_base_address, 0x200000)

.flashMailbox
 *(.flashMailbox)
                0x0000000000201000                PROVIDE (_tlv_base_address, 0x201000)

.tlvTable
 *(.tlvTable)
                0x0000000000202000                PROVIDE (_bsl_base_address, 0x202000)

.bslArea
 *(.bslArea)
                0x0000000020000000                PROVIDE (_vtable_base_address, DEFINED (_vtable_base_address)?_vtable_base_address:0x20000000)

.vtable
 *(.vtable)

.text           0x00000000000000e4     0x1e1c
 CREATE_OBJECT_SYMBOLS
 *(.text)
 .text          0x00000000000000e4        0x0 /opt/ti/ccsv7/tools/compiler/gcc-arm-none-eabi-6-2017-q1-update/bin/../lib/gcc/arm-none-eabi/6.3.1/thumb/v7e-m/fpv4-sp/hard/crti.o
 .text          0x00000000000000e4       0x6c /opt/ti/ccsv7/tools/compiler/gcc-arm-none-eabi-6-2017-q1-update/bin/../lib/gcc/arm-none-eabi/6.3.1/thumb/v7e-m/fpv4-sp/hard/crtbegin.o
 .text          0x0000000000000150       0x74 /opt/ti/ccsv7/tools/compiler/gcc-arm-none-eabi-6-2017-q1-update/bin/../lib/gcc/arm-none-eabi/6.3.1/../../../../arm-none-eabi/lib/thumb/v7e-m/fpv4-sp/hard/crt0.o
                0x0000000000000150                _mainCRTStartup
                0x0000000000000150                _start
 .text          0x00000000000001c4        0x0 /opt/ti/ccsv7/tools/compiler/gcc-arm-none-eabi-6-2017-q1-update/bin/../lib/gcc/arm-none-eabi/6.3.1/../../../../arm-none-eabi/lib/thumb/v7e-m/fpv4-sp/hard/libc_nano.a(lib_a-exit.o)
 .text          0x00000000000001c4        0x0 /opt/ti/ccsv7/tools/compiler/gcc-arm-none-eabi-6-2017-q1-update/bin/../lib/gcc/arm-none-eabi/6.3.1/../../../../arm-none-eabi/lib/thumb/v7e-m/fpv4-sp/hard/libc_nano.a(lib_a-impure.o)
 .text          0x00000000000001c4        0x0 /opt/ti/ccsv7/tools/compiler/gcc-arm-none-eabi-6-2017-q1-update/bin/../lib/gcc/arm-none-eabi/6.3.1/../../../../arm-none-eabi/lib/thumb/v7e-m/fpv4-sp/hard/libc_nano.a(lib_a-init.o)
 .text          0x00000000000001c4        0x0 /opt/ti/ccsv7/tools/compiler/gcc-arm-none-eabi-6-2017-q1-update/bin/../lib/gcc/arm-none-eabi/6.3.1/../../../../arm-none-eabi/lib/thumb/v7e-m/fpv4-sp/hard/libc_nano.a(lib_a-memset.o)
 .text          0x00000000000001c4        0x0 /opt/ti/ccsv7/tools/compiler/gcc-arm-none-eabi-6-2017-q1-update/bin/../lib/gcc/arm-none-eabi/6.3.1/../../../../arm-none-eabi/lib/thumb/v7e-m/fpv4-sp/hard/libnosys.a(_exit.o)
 .text          0x00000000000001c4        0x0 Debug/main.cpp.o
 .text          0x00000000000001c4        0x0 Debug/startup_msp432p401r_gcc.c.o
 .text          0x00000000000001c4        0x0 Debug/system_msp432p401r.c.o
 .text          0x00000000000001c4        0x0 /home/student/git/workspace_mct/YAHAL/libYAHAL_msp432.a(gpio_msp432.cpp.o)
 .text          0x00000000000001c4        0x0 /home/student/git/workspace_mct/YAHAL/libYAHAL_msp432.a(timer_msp432.cpp.o)
 .text          0x00000000000001c4        0x0 /opt/ti/ccsv7/tools/compiler/gcc-arm-none-eabi-6-2017-q1-update/bin/../lib/gcc/arm-none-eabi/6.3.1/../../../../arm-none-eabi/lib/thumb/v7e-m/fpv4-sp/hard/libstdc++_nano.a(class_type_info.o)
 .text          0x00000000000001c4        0x0 /opt/ti/ccsv7/tools/compiler/gcc-arm-none-eabi-6-2017-q1-update/bin/../lib/gcc/arm-none-eabi/6.3.1/../../../../arm-none-eabi/lib/thumb/v7e-m/fpv4-sp/hard/libstdc++_nano.a(atexit_arm.o)
 .text          0x00000000000001c4        0x0 /opt/ti/ccsv7/tools/compiler/gcc-arm-none-eabi-6-2017-q1-update/bin/../lib/gcc/arm-none-eabi/6.3.1/../../../../arm-none-eabi/lib/thumb/v7e-m/fpv4-sp/hard/libstdc++_nano.a(si_class_type_info.o)
 .text          0x00000000000001c4        0x0 /opt/ti/ccsv7/tools/compiler/gcc-arm-none-eabi-6-2017-q1-update/bin/../lib/gcc/arm-none-eabi/6.3.1/../../../../arm-none-eabi/lib/thumb/v7e-m/fpv4-sp/hard/libstdc++_nano.a(del_ops.o)
 .text          0x00000000000001c4        0x0 /opt/ti/ccsv7/tools/compiler/gcc-arm-none-eabi-6-2017-q1-update/bin/../lib/gcc/arm-none-eabi/6.3.1/../../../../arm-none-eabi/lib/thumb/v7e-m/fpv4-sp/hard/libstdc++_nano.a(del_op.o)
 .text          0x00000000000001c4        0x0 /opt/ti/ccsv7/tools/compiler/gcc-arm-none-eabi-6-2017-q1-update/bin/../lib/gcc/arm-none-eabi/6.3.1/../../../../arm-none-eabi/lib/thumb/v7e-m/fpv4-sp/hard/libstdc++_nano.a(pure.o)
 .text          0x00000000000001c4        0x0 /opt/ti/ccsv7/tools/compiler/gcc-arm-none-eabi-6-2017-q1-update/bin/../lib/gcc/arm-none-eabi/6.3.1/../../../../arm-none-eabi/lib/thumb/v7e-m/fpv4-sp/hard/libstdc++_nano.a(tinfo.o)
 .text          0x00000000000001c4        0x0 /opt/ti/ccsv7/tools/compiler/gcc-arm-none-eabi-6-2017-q1-update/bin/../lib/gcc/arm-none-eabi/6.3.1/../../../../arm-none-eabi/lib/thumb/v7e-m/fpv4-sp/hard/libstdc++_nano.a(eh_terminate.o)
 .text          0x00000000000001c4        0x0 /opt/ti/ccsv7/tools/compiler/gcc-arm-none-eabi-6-2017-q1-update/bin/../lib/gcc/arm-none-eabi/6.3.1/../../../../arm-none-eabi/lib/thumb/v7e-m/fpv4-sp/hard/libstdc++_nano.a(eh_term_handler.o)
 .text          0x00000000000001c4        0x0 /opt/ti/ccsv7/tools/compiler/gcc-arm-none-eabi-6-2017-q1-update/bin/../lib/gcc/arm-none-eabi/6.3.1/../../../../arm-none-eabi/lib/thumb/v7e-m/fpv4-sp/hard/libstdc++_nano.a(eh_unex_handler.o)
 .text          0x00000000000001c4        0x0 /opt/ti/ccsv7/tools/compiler/gcc-arm-none-eabi-6-2017-q1-update/bin/../lib/gcc/arm-none-eabi/6.3.1/../../../../arm-none-eabi/lib/thumb/v7e-m/fpv4-sp/hard/libc_nano.a(lib_a-abort.o)
 .text          0x00000000000001c4        0x0 /opt/ti/ccsv7/tools/compiler/gcc-arm-none-eabi-6-2017-q1-update/bin/../lib/gcc/arm-none-eabi/6.3.1/../../../../arm-none-eabi/lib/thumb/v7e-m/fpv4-sp/hard/libc_nano.a(lib_a-cxa_atexit.o)
 .text          0x00000000000001c4        0x0 /opt/ti/ccsv7/tools/compiler/gcc-arm-none-eabi-6-2017-q1-update/bin/../lib/gcc/arm-none-eabi/6.3.1/../../../../arm-none-eabi/lib/thumb/v7e-m/fpv4-sp/hard/libc_nano.a(lib_a-malloc.o)
 .text          0x00000000000001c4        0x0 /opt/ti/ccsv7/tools/compiler/gcc-arm-none-eabi-6-2017-q1-update/bin/../lib/gcc/arm-none-eabi/6.3.1/../../../../arm-none-eabi/lib/thumb/v7e-m/fpv4-sp/hard/libc_nano.a(lib_a-nano-freer.o)
 .text          0x00000000000001c4        0x0 /opt/ti/ccsv7/tools/compiler/gcc-arm-none-eabi-6-2017-q1-update/bin/../lib/gcc/arm-none-eabi/6.3.1/../../../../arm-none-eabi/lib/thumb/v7e-m/fpv4-sp/hard/libc_nano.a(lib_a-nano-mallocr.o)
 .text          0x00000000000001c4        0x0 /opt/ti/ccsv7/tools/compiler/gcc-arm-none-eabi-6-2017-q1-update/bin/../lib/gcc/arm-none-eabi/6.3.1/../../../../arm-none-eabi/lib/thumb/v7e-m/fpv4-sp/hard/libc_nano.a(lib_a-on_exit_args.o)
 .text          0x00000000000001c4        0x0 /opt/ti/ccsv7/tools/compiler/gcc-arm-none-eabi-6-2017-q1-update/bin/../lib/gcc/arm-none-eabi/6.3.1/../../../../arm-none-eabi/lib/thumb/v7e-m/fpv4-sp/hard/libc_nano.a(lib_a-sbrkr.o)
 .text          0x00000000000001c4        0x0 /opt/ti/ccsv7/tools/compiler/gcc-arm-none-eabi-6-2017-q1-update/bin/../lib/gcc/arm-none-eabi/6.3.1/../../../../arm-none-eabi/lib/thumb/v7e-m/fpv4-sp/hard/libc_nano.a(lib_a-signal.o)
 .text          0x00000000000001c4        0x0 /opt/ti/ccsv7/tools/compiler/gcc-arm-none-eabi-6-2017-q1-update/bin/../lib/gcc/arm-none-eabi/6.3.1/../../../../arm-none-eabi/lib/thumb/v7e-m/fpv4-sp/hard/libc_nano.a(lib_a-signalr.o)
 .text          0x00000000000001c4       0x14 /opt/ti/ccsv7/tools/compiler/gcc-arm-none-eabi-6-2017-q1-update/bin/../lib/gcc/arm-none-eabi/6.3.1/../../../../arm-none-eabi/lib/thumb/v7e-m/fpv4-sp/hard/libc_nano.a(lib_a-strcmp.o)
                0x00000000000001c4                strcmp
 .text          0x00000000000001d8        0x0 /opt/ti/ccsv7/tools/compiler/gcc-arm-none-eabi-6-2017-q1-update/bin/../lib/gcc/arm-none-eabi/6.3.1/../../../../arm-none-eabi/lib/thumb/v7e-m/fpv4-sp/hard/libc_nano.a(lib_a-mlock.o)
 .text          0x00000000000001d8        0x0 /opt/ti/ccsv7/tools/compiler/gcc-arm-none-eabi-6-2017-q1-update/bin/../lib/gcc/arm-none-eabi/6.3.1/../../../../arm-none-eabi/lib/thumb/v7e-m/fpv4-sp/hard/libc_nano.a(lib_a-reent.o)
 .text          0x00000000000001d8        0x0 /opt/ti/ccsv7/tools/compiler/gcc-arm-none-eabi-6-2017-q1-update/bin/../lib/gcc/arm-none-eabi/6.3.1/../../../../arm-none-eabi/lib/thumb/v7e-m/fpv4-sp/hard/libnosys.a(getpid.o)
 .text          0x00000000000001d8        0x0 /opt/ti/ccsv7/tools/compiler/gcc-arm-none-eabi-6-2017-q1-update/bin/../lib/gcc/arm-none-eabi/6.3.1/../../../../arm-none-eabi/lib/thumb/v7e-m/fpv4-sp/hard/libnosys.a(kill.o)
 .text          0x00000000000001d8        0x0 /opt/ti/ccsv7/tools/compiler/gcc-arm-none-eabi-6-2017-q1-update/bin/../lib/gcc/arm-none-eabi/6.3.1/../../../../arm-none-eabi/lib/thumb/v7e-m/fpv4-sp/hard/libnosys.a(sbrk.o)
 .text          0x00000000000001d8        0x0 /opt/ti/ccsv7/tools/compiler/gcc-arm-none-eabi-6-2017-q1-update/bin/../lib/gcc/arm-none-eabi/6.3.1/thumb/v7e-m/fpv4-sp/hard/crtend.o
 .text          0x00000000000001d8        0x0 /opt/ti/ccsv7/tools/compiler/gcc-arm-none-eabi-6-2017-q1-update/bin/../lib/gcc/arm-none-eabi/6.3.1/thumb/v7e-m/fpv4-sp/hard/crtn.o
 *(.text.*)
 .text.exit     0x00000000000001d8       0x28 /opt/ti/ccsv7/tools/compiler/gcc-arm-none-eabi-6-2017-q1-update/bin/../lib/gcc/arm-none-eabi/6.3.1/../../../../arm-none-eabi/lib/thumb/v7e-m/fpv4-sp/hard/libc_nano.a(lib_a-exit.o)
                0x00000000000001d8                exit
 .text.__libc_init_array
                0x0000000000000200       0x48 /opt/ti/ccsv7/tools/compiler/gcc-arm-none-eabi-6-2017-q1-update/bin/../lib/gcc/arm-none-eabi/6.3.1/../../../../arm-none-eabi/lib/thumb/v7e-m/fpv4-sp/hard/libc_nano.a(lib_a-init.o)
                0x0000000000000200                __libc_init_array
 .text.memset   0x0000000000000248       0x10 /opt/ti/ccsv7/tools/compiler/gcc-arm-none-eabi-6-2017-q1-update/bin/../lib/gcc/arm-none-eabi/6.3.1/../../../../arm-none-eabi/lib/thumb/v7e-m/fpv4-sp/hard/libc_nano.a(lib_a-memset.o)
                0x0000000000000248                memset
 .text._exit    0x0000000000000258        0x4 /opt/ti/ccsv7/tools/compiler/gcc-arm-none-eabi-6-2017-q1-update/bin/../lib/gcc/arm-none-eabi/6.3.1/../../../../arm-none-eabi/lib/thumb/v7e-m/fpv4-sp/hard/libnosys.a(_exit.o)
                0x0000000000000258                _exit
 .text._ZN8gpio_pinC2ER14gpio_interfacet
                0x000000000000025c       0x28 Debug/main.cpp.o
                0x000000000000025c                gpio_pin::gpio_pin(gpio_interface&, unsigned short)
                0x000000000000025c                gpio_pin::gpio_pin(gpio_interface&, unsigned short)
 .text._ZN8gpio_pin8gpioModeEt
                0x0000000000000284       0x28 Debug/main.cpp.o
                0x0000000000000284                gpio_pin::gpioMode(unsigned short)
 .text._ZN8gpio_pin9gpioWriteEb
                0x00000000000002ac       0x2a Debug/main.cpp.o
                0x00000000000002ac                gpio_pin::gpioWrite(bool)
 .text._ZN8gpio_pin10gpioToggleEv
                0x00000000000002d6       0x26 Debug/main.cpp.o
                0x00000000000002d6                gpio_pin::gpioToggle()
 .text._ZN15gpio_msp432_pinC2Et
                0x00000000000002fc       0x28 Debug/main.cpp.o
                0x00000000000002fc                gpio_msp432_pin::gpio_msp432_pin(unsigned short)
                0x00000000000002fc                gpio_msp432_pin::gpio_msp432_pin(unsigned short)
 .text._Z9callback1Pv
                0x0000000000000324       0x1c Debug/main.cpp.o
                0x0000000000000324                callback1(void*)
 .text._Z9callback2Pv
                0x0000000000000340       0x1a Debug/main.cpp.o
                0x0000000000000340                callback2(void*)
 *fill*         0x000000000000035a        0x2 
 .text._Z5delayi
                0x000000000000035c       0x64 Debug/main.cpp.o
                0x000000000000035c                delay(int)
 .text.main     0x00000000000003c0       0xb8 Debug/main.cpp.o
                0x00000000000003c0                main
 .text.Reset_Handler
                0x0000000000000478       0x44 Debug/startup_msp432p401r_gcc.c.o
                0x0000000000000478                Reset_Handler
 .text.Default_Handler
                0x00000000000004bc        0x6 Debug/startup_msp432p401r_gcc.c.o
                0x00000000000004bc                CS_IRQHandler
                0x00000000000004bc                DebugMon_Handler
                0x00000000000004bc                AES256_IRQHandler
                0x00000000000004bc                HardFault_Handler
                0x00000000000004bc                SysTick_Handler
                0x00000000000004bc                PendSV_Handler
                0x00000000000004bc                NMI_Handler
                0x00000000000004bc                RTC_C_IRQHandler
                0x00000000000004bc                FPU_IRQHandler
                0x00000000000004bc                TA3_0_IRQHandler
                0x00000000000004bc                UsageFault_Handler
                0x00000000000004bc                DMA_INT3_IRQHandler
                0x00000000000004bc                TA2_0_IRQHandler
                0x00000000000004bc                DMA_INT1_IRQHandler
                0x00000000000004bc                WDT_A_IRQHandler
                0x00000000000004bc                TA2_N_IRQHandler
                0x00000000000004bc                TA1_0_IRQHandler
                0x00000000000004bc                PSS_IRQHandler
                0x00000000000004bc                DMA_INT2_IRQHandler
                0x00000000000004bc                EUSCIA3_IRQHandler
                0x00000000000004bc                DMA_INT0_IRQHandler
                0x00000000000004bc                EUSCIB0_IRQHandler
                0x00000000000004bc                Default_Handler
                0x00000000000004bc                T32_INTC_IRQHandler
                0x00000000000004bc                TA3_N_IRQHandler
                0x00000000000004bc                TA0_0_IRQHandler
                0x00000000000004bc                EUSCIA2_IRQHandler
                0x00000000000004bc                MemManage_Handler
                0x00000000000004bc                SVC_Handler
                0x00000000000004bc                TA1_N_IRQHandler
                0x00000000000004bc                EUSCIA1_IRQHandler
                0x00000000000004bc                COMP_E1_IRQHandler
                0x00000000000004bc                EUSCIB2_IRQHandler
                0x00000000000004bc                FLCTL_IRQHandler
                0x00000000000004bc                EUSCIB3_IRQHandler
                0x00000000000004bc                DMA_ERR_IRQHandler
                0x00000000000004bc                ADC14_IRQHandler
                0x00000000000004bc                EUSCIA0_IRQHandler
                0x00000000000004bc                BusFault_Handler
                0x00000000000004bc                PCM_IRQHandler
                0x00000000000004bc                TA0_N_IRQHandler
                0x00000000000004bc                COMP_E0_IRQHandler
                0x00000000000004bc                EUSCIB1_IRQHandler
 *fill*         0x00000000000004c2        0x2 
 .text.SystemCoreClockUpdate
                0x00000000000004c4      0x2f8 Debug/system_msp432p401r.c.o
                0x00000000000004c4                SystemCoreClockUpdate
 .text.SystemInit
                0x00000000000007bc       0x80 Debug/system_msp432p401r.c.o
                0x00000000000007bc                SystemInit
 .text.__NVIC_EnableIRQ
                0x000000000000083c       0x3c /home/student/git/workspace_mct/YAHAL/libYAHAL_msp432.a(gpio_msp432.cpp.o)
 .text._ZN14gpio_interfaceD2Ev
                0x0000000000000878       0x20 /home/student/git/workspace_mct/YAHAL/libYAHAL_msp432.a(gpio_msp432.cpp.o)
                0x0000000000000878                gpio_interface::~gpio_interface()
                0x0000000000000878                gpio_interface::~gpio_interface()
 .text._ZN14gpio_interfaceD0Ev
                0x0000000000000898       0x1e /home/student/git/workspace_mct/YAHAL/libYAHAL_msp432.a(gpio_msp432.cpp.o)
                0x0000000000000898                gpio_interface::~gpio_interface()
 *fill*         0x00000000000008b6        0x2 
 .text._ZN11gpio_msp432D2Ev
                0x00000000000008b8       0x24 /home/student/git/workspace_mct/YAHAL/libYAHAL_msp432.a(gpio_msp432.cpp.o)
                0x00000000000008b8                gpio_msp432::~gpio_msp432()
                0x00000000000008b8                gpio_msp432::~gpio_msp432()
 .text._ZN11gpio_msp432D0Ev
                0x00000000000008dc       0x1e /home/student/git/workspace_mct/YAHAL/libYAHAL_msp432.a(gpio_msp432.cpp.o)
                0x00000000000008dc                gpio_msp432::~gpio_msp432()
 *fill*         0x00000000000008fa        0x2 
 .text._ZN14gpio_interfaceC2Ev
                0x00000000000008fc       0x20 /home/student/git/workspace_mct/YAHAL/libYAHAL_msp432.a(gpio_msp432.cpp.o)
                0x00000000000008fc                gpio_interface::gpio_interface()
                0x00000000000008fc                gpio_interface::gpio_interface()
 .text._ZN11gpio_msp432C2Ev
                0x000000000000091c       0x24 /home/student/git/workspace_mct/YAHAL/libYAHAL_msp432.a(gpio_msp432.cpp.o)
                0x000000000000091c                gpio_msp432::gpio_msp432()
                0x000000000000091c                gpio_msp432::gpio_msp432()
 .text._ZL17yahal_assert_funcv
                0x0000000000000940       0x1c /home/student/git/workspace_mct/YAHAL/libYAHAL_msp432.a(gpio_msp432.cpp.o)
 .text._ZN11gpio_msp4328gpioModeEtt
                0x000000000000095c       0x30 /home/student/git/workspace_mct/YAHAL/libYAHAL_msp432.a(gpio_msp432.cpp.o)
                0x000000000000095c                gpio_msp432::gpioMode(unsigned short, unsigned short)
 .text._ZN11gpio_msp4328gpioReadEt
                0x000000000000098c       0x70 /home/student/git/workspace_mct/YAHAL/libYAHAL_msp432.a(gpio_msp432.cpp.o)
                0x000000000000098c                gpio_msp432::gpioRead(unsigned short)
 .text._ZN11gpio_msp4329gpioWriteEtb
                0x00000000000009fc      0x1d4 /home/student/git/workspace_mct/YAHAL/libYAHAL_msp432.a(gpio_msp432.cpp.o)
                0x00000000000009fc                gpio_msp432::gpioWrite(unsigned short, bool)
 .text._ZN11gpio_msp43210gpioToggleEt
                0x0000000000000bd0       0x7c /home/student/git/workspace_mct/YAHAL/libYAHAL_msp432.a(gpio_msp432.cpp.o)
                0x0000000000000bd0                gpio_msp432::gpioToggle(unsigned short)
 .text._ZN11gpio_msp43213gpioAttachIrqEtPFvtEt
                0x0000000000000c4c       0xf8 /home/student/git/workspace_mct/YAHAL/libYAHAL_msp432.a(gpio_msp432.cpp.o)
                0x0000000000000c4c                gpio_msp432::gpioAttachIrq(unsigned short, void (*)(unsigned short), unsigned short)
 .text._ZN11gpio_msp43213gpioDetachIrqEt
                0x0000000000000d44       0x70 /home/student/git/workspace_mct/YAHAL/libYAHAL_msp432.a(gpio_msp432.cpp.o)
                0x0000000000000d44                gpio_msp432::gpioDetachIrq(unsigned short)
 .text._ZN11gpio_msp43213gpioEnableIrqEt
                0x0000000000000db4       0x78 /home/student/git/workspace_mct/YAHAL/libYAHAL_msp432.a(gpio_msp432.cpp.o)
                0x0000000000000db4                gpio_msp432::gpioEnableIrq(unsigned short)
 .text._ZN11gpio_msp43214gpioDisableIrqEt
                0x0000000000000e2c       0x68 /home/student/git/workspace_mct/YAHAL/libYAHAL_msp432.a(gpio_msp432.cpp.o)
                0x0000000000000e2c                gpio_msp432::gpioDisableIrq(unsigned short)
 .text._ZN11gpio_msp4329handleIrqEhh
                0x0000000000000e94       0x3e /home/student/git/workspace_mct/YAHAL/libYAHAL_msp432.a(gpio_msp432.cpp.o)
                0x0000000000000e94                gpio_msp432::handleIrq(unsigned char, unsigned char)
 *fill*         0x0000000000000ed2        0x2 
 .text._ZN11gpio_msp4326setSELEth
                0x0000000000000ed4       0x94 /home/student/git/workspace_mct/YAHAL/libYAHAL_msp432.a(gpio_msp432.cpp.o)
                0x0000000000000ed4                gpio_msp432::setSEL(unsigned short, unsigned char)
 .text._ZN11gpio_msp4327setModeEtt
                0x0000000000000f68      0x2f4 /home/student/git/workspace_mct/YAHAL/libYAHAL_msp432.a(gpio_msp432.cpp.o)
                0x0000000000000f68                gpio_msp432::setMode(unsigned short, unsigned short)
 .text.PORT1_IRQHandler
                0x000000000000125c       0x44 /home/student/git/workspace_mct/YAHAL/libYAHAL_msp432.a(gpio_msp432.cpp.o)
                0x000000000000125c                PORT1_IRQHandler
 .text.PORT2_IRQHandler
                0x00000000000012a0       0x44 /home/student/git/workspace_mct/YAHAL/libYAHAL_msp432.a(gpio_msp432.cpp.o)
                0x00000000000012a0                PORT2_IRQHandler
 .text.PORT3_IRQHandler
                0x00000000000012e4       0x44 /home/student/git/workspace_mct/YAHAL/libYAHAL_msp432.a(gpio_msp432.cpp.o)
                0x00000000000012e4                PORT3_IRQHandler
 .text.PORT4_IRQHandler
                0x0000000000001328       0x44 /home/student/git/workspace_mct/YAHAL/libYAHAL_msp432.a(gpio_msp432.cpp.o)
                0x0000000000001328                PORT4_IRQHandler
 .text.PORT5_IRQHandler
                0x000000000000136c       0x44 /home/student/git/workspace_mct/YAHAL/libYAHAL_msp432.a(gpio_msp432.cpp.o)
                0x000000000000136c                PORT5_IRQHandler
 .text.PORT6_IRQHandler
                0x00000000000013b0       0x44 /home/student/git/workspace_mct/YAHAL/libYAHAL_msp432.a(gpio_msp432.cpp.o)
                0x00000000000013b0                PORT6_IRQHandler
 .text._Z41__static_initialization_and_destruction_0ii
                0x00000000000013f4       0x40 /home/student/git/workspace_mct/YAHAL/libYAHAL_msp432.a(gpio_msp432.cpp.o)
 .text._GLOBAL__sub_I_port_base
                0x0000000000001434       0x10 /home/student/git/workspace_mct/YAHAL/libYAHAL_msp432.a(gpio_msp432.cpp.o)
 .text.__NVIC_EnableIRQ
                0x0000000000001444       0x3c /home/student/git/workspace_mct/YAHAL/libYAHAL_msp432.a(timer_msp432.cpp.o)
 .text._ZL17yahal_assert_funcv
                0x0000000000001480       0x1c /home/student/git/workspace_mct/YAHAL/libYAHAL_msp432.a(timer_msp432.cpp.o)
 .text._ZN15timer_interfaceC2Ev
                0x000000000000149c       0x20 /home/student/git/workspace_mct/YAHAL/libYAHAL_msp432.a(timer_msp432.cpp.o)
                0x000000000000149c                timer_interface::timer_interface()
                0x000000000000149c                timer_interface::timer_interface()
 .text._ZN15timer_interfaceD2Ev
                0x00000000000014bc       0x20 /home/student/git/workspace_mct/YAHAL/libYAHAL_msp432.a(timer_msp432.cpp.o)
                0x00000000000014bc                timer_interface::~timer_interface()
                0x00000000000014bc                timer_interface::~timer_interface()
 .text._ZN15timer_interfaceD0Ev
                0x00000000000014dc       0x1e /home/student/git/workspace_mct/YAHAL/libYAHAL_msp432.a(timer_msp432.cpp.o)
                0x00000000000014dc                timer_interface::~timer_interface()
 *fill*         0x00000000000014fa        0x2 
 .text._ZN12timer_msp432C2EP12Timer32_Type
                0x00000000000014fc       0x70 /home/student/git/workspace_mct/YAHAL/libYAHAL_msp432.a(timer_msp432.cpp.o)
                0x00000000000014fc                timer_msp432::timer_msp432(Timer32_Type*)
                0x00000000000014fc                timer_msp432::timer_msp432(Timer32_Type*)
 .text._ZN12timer_msp432D2Ev
                0x000000000000156c       0x2c /home/student/git/workspace_mct/YAHAL/libYAHAL_msp432.a(timer_msp432.cpp.o)
                0x000000000000156c                timer_msp432::~timer_msp432()
                0x000000000000156c                timer_msp432::~timer_msp432()
 .text._ZN12timer_msp432D0Ev
                0x0000000000001598       0x1e /home/student/git/workspace_mct/YAHAL/libYAHAL_msp432.a(timer_msp432.cpp.o)
                0x0000000000001598                timer_msp432::~timer_msp432()
 .text._ZN12timer_msp4329setPeriodEmN5TIMER10timer_modeE
                0x00000000000015b6       0x60 /home/student/git/workspace_mct/YAHAL/libYAHAL_msp432.a(timer_msp432.cpp.o)
                0x00000000000015b6                timer_msp432::setPeriod(unsigned long, TIMER::timer_mode)
 .text._ZN12timer_msp4329getPeriodEv
                0x0000000000001616       0x18 /home/student/git/workspace_mct/YAHAL/libYAHAL_msp432.a(timer_msp432.cpp.o)
                0x0000000000001616                timer_msp432::getPeriod()
 *fill*         0x000000000000162e        0x2 
 .text._ZN12timer_msp43211setCallbackEPFvPvES0_
                0x0000000000001630       0x50 /home/student/git/workspace_mct/YAHAL/libYAHAL_msp432.a(timer_msp432.cpp.o)
                0x0000000000001630                timer_msp432::setCallback(void (*)(void*), void*)
 .text._ZN12timer_msp4325startEv
                0x0000000000001680       0x24 /home/student/git/workspace_mct/YAHAL/libYAHAL_msp432.a(timer_msp432.cpp.o)
                0x0000000000001680                timer_msp432::start()
 .text._ZN12timer_msp4324stopEv
                0x00000000000016a4       0x24 /home/student/git/workspace_mct/YAHAL/libYAHAL_msp432.a(timer_msp432.cpp.o)
                0x00000000000016a4                timer_msp432::stop()
 .text._ZN12timer_msp4329isRunningEv
                0x00000000000016c8       0x28 /home/student/git/workspace_mct/YAHAL/libYAHAL_msp432.a(timer_msp432.cpp.o)
                0x00000000000016c8                timer_msp432::isRunning()
 .text._ZN12timer_msp43210getCounterEv
                0x00000000000016f0       0x28 /home/student/git/workspace_mct/YAHAL/libYAHAL_msp432.a(timer_msp432.cpp.o)
                0x00000000000016f0                timer_msp432::getCounter()
 .text._ZN12timer_msp43212resetCounterEv
                0x0000000000001718       0x1e /home/student/git/workspace_mct/YAHAL/libYAHAL_msp432.a(timer_msp432.cpp.o)
                0x0000000000001718                timer_msp432::resetCounter()
 *fill*         0x0000000000001736        0x2 
 .text.T32_INT1_IRQHandler
                0x0000000000001738       0x50 /home/student/git/workspace_mct/YAHAL/libYAHAL_msp432.a(timer_msp432.cpp.o)
                0x0000000000001738                T32_INT1_IRQHandler
 .text.T32_INT2_IRQHandler
                0x0000000000001788       0x50 /home/student/git/workspace_mct/YAHAL/libYAHAL_msp432.a(timer_msp432.cpp.o)
                0x0000000000001788                T32_INT2_IRQHandler
 .text._ZNK10__cxxabiv117__class_type_info11__do_upcastEPKS0_PPv
                0x00000000000017d8       0x34 /opt/ti/ccsv7/tools/compiler/gcc-arm-none-eabi-6-2017-q1-update/bin/../lib/gcc/arm-none-eabi/6.3.1/../../../../arm-none-eabi/lib/thumb/v7e-m/fpv4-sp/hard/libstdc++_nano.a(class_type_info.o)
                0x00000000000017d8                __cxxabiv1::__class_type_info::__do_upcast(__cxxabiv1::__class_type_info const*, void**) const
 .text._ZNK10__cxxabiv117__class_type_info20__do_find_public_srcEiPKvPKS0_S2_
                0x000000000000180c        0xc /opt/ti/ccsv7/tools/compiler/gcc-arm-none-eabi-6-2017-q1-update/bin/../lib/gcc/arm-none-eabi/6.3.1/../../../../arm-none-eabi/lib/thumb/v7e-m/fpv4-sp/hard/libstdc++_nano.a(class_type_info.o)
                0x000000000000180c                __cxxabiv1::__class_type_info::__do_find_public_src(int, void const*, __cxxabiv1::__class_type_info const*, void const*) const
 .text._ZN10__cxxabiv117__class_type_infoD2Ev
                0x0000000000001818       0x14 /opt/ti/ccsv7/tools/compiler/gcc-arm-none-eabi-6-2017-q1-update/bin/../lib/gcc/arm-none-eabi/6.3.1/../../../../arm-none-eabi/lib/thumb/v7e-m/fpv4-sp/hard/libstdc++_nano.a(class_type_info.o)
                0x0000000000001818                __cxxabiv1::__class_type_info::~__class_type_info()
                0x0000000000001818                __cxxabiv1::__class_type_info::~__class_type_info()
 .text._ZN10__cxxabiv117__class_type_infoD0Ev
                0x000000000000182c       0x14 /opt/ti/ccsv7/tools/compiler/gcc-arm-none-eabi-6-2017-q1-update/bin/../lib/gcc/arm-none-eabi/6.3.1/../../../../arm-none-eabi/lib/thumb/v7e-m/fpv4-sp/hard/libstdc++_nano.a(class_type_info.o)
                0x000000000000182c                __cxxabiv1::__class_type_info::~__class_type_info()
 .text._ZNK10__cxxabiv117__class_type_info11__do_upcastEPKS0_PKvRNS0_15__upcast_resultE
                0x0000000000001840       0x18 /opt/ti/ccsv7/tools/compiler/gcc-arm-none-eabi-6-2017-q1-update/bin/../lib/gcc/arm-none-eabi/6.3.1/../../../../arm-none-eabi/lib/thumb/v7e-m/fpv4-sp/hard/libstdc++_nano.a(class_type_info.o)
                0x0000000000001840                __cxxabiv1::__class_type_info::__do_upcast(__cxxabiv1::__class_type_info const*, void const*, __cxxabiv1::__class_type_info::__upcast_result&) const
 .text._ZNK10__cxxabiv117__class_type_info10__do_catchEPKSt9type_infoPPvj
                0x0000000000001858       0x2a /opt/ti/ccsv7/tools/compiler/gcc-arm-none-eabi-6-2017-q1-update/bin/../lib/gcc/arm-none-eabi/6.3.1/../../../../arm-none-eabi/lib/thumb/v7e-m/fpv4-sp/hard/libstdc++_nano.a(class_type_info.o)
                0x0000000000001858                __cxxabiv1::__class_type_info::__do_catch(std::type_info const*, void**, unsigned int) const
 .text._ZNK10__cxxabiv117__class_type_info12__do_dyncastEiNS0_10__sub_kindEPKS0_PKvS3_S5_RNS0_16__dyncast_resultE
                0x0000000000001882       0x38 /opt/ti/ccsv7/tools/compiler/gcc-arm-none-eabi-6-2017-q1-update/bin/../lib/gcc/arm-none-eabi/6.3.1/../../../../arm-none-eabi/lib/thumb/v7e-m/fpv4-sp/hard/libstdc++_nano.a(class_type_info.o)
                0x0000000000001882                __cxxabiv1::__class_type_info::__do_dyncast(int, __cxxabiv1::__class_type_info::__sub_kind, __cxxabiv1::__class_type_info const*, void const*, __cxxabiv1::__class_type_info const*, void const*, __cxxabiv1::__class_type_info::__dyncast_result&) const
 .text.__aeabi_atexit
                0x00000000000018ba        0xa /opt/ti/ccsv7/tools/compiler/gcc-arm-none-eabi-6-2017-q1-update/bin/../lib/gcc/arm-none-eabi/6.3.1/../../../../arm-none-eabi/lib/thumb/v7e-m/fpv4-sp/hard/libstdc++_nano.a(atexit_arm.o)
                0x00000000000018ba                __aeabi_atexit
 .text._ZN10__cxxabiv120__si_class_type_infoD2Ev
                0x00000000000018c4       0x14 /opt/ti/ccsv7/tools/compiler/gcc-arm-none-eabi-6-2017-q1-update/bin/../lib/gcc/arm-none-eabi/6.3.1/../../../../arm-none-eabi/lib/thumb/v7e-m/fpv4-sp/hard/libstdc++_nano.a(si_class_type_info.o)
                0x00000000000018c4                __cxxabiv1::__si_class_type_info::~__si_class_type_info()
                0x00000000000018c4                __cxxabiv1::__si_class_type_info::~__si_class_type_info()
 .text._ZN10__cxxabiv120__si_class_type_infoD0Ev
                0x00000000000018d8       0x14 /opt/ti/ccsv7/tools/compiler/gcc-arm-none-eabi-6-2017-q1-update/bin/../lib/gcc/arm-none-eabi/6.3.1/../../../../arm-none-eabi/lib/thumb/v7e-m/fpv4-sp/hard/libstdc++_nano.a(si_class_type_info.o)
                0x00000000000018d8                __cxxabiv1::__si_class_type_info::~__si_class_type_info()
 .text._ZNK10__cxxabiv120__si_class_type_info20__do_find_public_srcEiPKvPKNS_17__class_type_infoES2_
                0x00000000000018ec       0x38 /opt/ti/ccsv7/tools/compiler/gcc-arm-none-eabi-6-2017-q1-update/bin/../lib/gcc/arm-none-eabi/6.3.1/../../../../arm-none-eabi/lib/thumb/v7e-m/fpv4-sp/hard/libstdc++_nano.a(si_class_type_info.o)
                0x00000000000018ec                __cxxabiv1::__si_class_type_info::__do_find_public_src(int, void const*, __cxxabiv1::__class_type_info const*, void const*) const
 .text._ZNK10__cxxabiv120__si_class_type_info12__do_dyncastEiNS_17__class_type_info10__sub_kindEPKS1_PKvS4_S6_RNS1_16__dyncast_resultE
                0x0000000000001924       0x7c /opt/ti/ccsv7/tools/compiler/gcc-arm-none-eabi-6-2017-q1-update/bin/../lib/gcc/arm-none-eabi/6.3.1/../../../../arm-none-eabi/lib/thumb/v7e-m/fpv4-sp/hard/libstdc++_nano.a(si_class_type_info.o)
                0x0000000000001924                __cxxabiv1::__si_class_type_info::__do_dyncast(int, __cxxabiv1::__class_type_info::__sub_kind, __cxxabiv1::__class_type_info const*, void const*, __cxxabiv1::__class_type_info const*, void const*, __cxxabiv1::__class_type_info::__dyncast_result&) const
 .text._ZNK10__cxxabiv120__si_class_type_info11__do_upcastEPKNS_17__class_type_infoEPKvRNS1_15__upcast_resultE
                0x00000000000019a0       0x2a /opt/ti/ccsv7/tools/compiler/gcc-arm-none-eabi-6-2017-q1-update/bin/../lib/gcc/arm-none-eabi/6.3.1/../../../../arm-none-eabi/lib/thumb/v7e-m/fpv4-sp/hard/libstdc++_nano.a(si_class_type_info.o)
                0x00000000000019a0                __cxxabiv1::__si_class_type_info::__do_upcast(__cxxabiv1::__class_type_info const*, void const*, __cxxabiv1::__class_type_info::__upcast_result&) const
 .text._ZdlPvj  0x00000000000019ca        0x4 /opt/ti/ccsv7/tools/compiler/gcc-arm-none-eabi-6-2017-q1-update/bin/../lib/gcc/arm-none-eabi/6.3.1/../../../../arm-none-eabi/lib/thumb/v7e-m/fpv4-sp/hard/libstdc++_nano.a(del_ops.o)
                0x00000000000019ca                operator delete(void*, unsigned int)
 .text._ZdlPv   0x00000000000019ce        0x4 /opt/ti/ccsv7/tools/compiler/gcc-arm-none-eabi-6-2017-q1-update/bin/../lib/gcc/arm-none-eabi/6.3.1/../../../../arm-none-eabi/lib/thumb/v7e-m/fpv4-sp/hard/libstdc++_nano.a(del_op.o)
                0x00000000000019ce                operator delete(void*)
 .text.__cxa_pure_virtual
                0x00000000000019d2        0x6 /opt/ti/ccsv7/tools/compiler/gcc-arm-none-eabi-6-2017-q1-update/bin/../lib/gcc/arm-none-eabi/6.3.1/../../../../arm-none-eabi/lib/thumb/v7e-m/fpv4-sp/hard/libstdc++_nano.a(pure.o)
                0x00000000000019d2                __cxa_pure_virtual
 .text.__cxa_deleted_virtual
                0x00000000000019d8        0x6 /opt/ti/ccsv7/tools/compiler/gcc-arm-none-eabi-6-2017-q1-update/bin/../lib/gcc/arm-none-eabi/6.3.1/../../../../arm-none-eabi/lib/thumb/v7e-m/fpv4-sp/hard/libstdc++_nano.a(pure.o)
                0x00000000000019d8                __cxa_deleted_virtual
 .text._ZNSt9type_infoD2Ev
                0x00000000000019de        0x2 /opt/ti/ccsv7/tools/compiler/gcc-arm-none-eabi-6-2017-q1-update/bin/../lib/gcc/arm-none-eabi/6.3.1/../../../../arm-none-eabi/lib/thumb/v7e-m/fpv4-sp/hard/libstdc++_nano.a(tinfo.o)
                0x00000000000019de                std::type_info::~type_info()
                0x00000000000019de                std::type_info::~type_info()
 .text._ZNKSt9type_info15__is_function_pEv
                0x00000000000019e0        0x4 /opt/ti/ccsv7/tools/compiler/gcc-arm-none-eabi-6-2017-q1-update/bin/../lib/gcc/arm-none-eabi/6.3.1/../../../../arm-none-eabi/lib/thumb/v7e-m/fpv4-sp/hard/libstdc++_nano.a(tinfo.o)
                0x00000000000019e0                std::type_info::__is_function_p() const
                0x00000000000019e0                std::type_info::__is_pointer_p() const
 .text._ZNKSt9type_info11__do_upcastEPKN10__cxxabiv117__class_type_infoEPPv
                0x00000000000019e4        0x4 /opt/ti/ccsv7/tools/compiler/gcc-arm-none-eabi-6-2017-q1-update/bin/../lib/gcc/arm-none-eabi/6.3.1/../../../../arm-none-eabi/lib/thumb/v7e-m/fpv4-sp/hard/libstdc++_nano.a(tinfo.o)
                0x00000000000019e4                std::type_info::__do_upcast(__cxxabiv1::__class_type_info const*, void**) const
 .text._ZNSt9type_infoD0Ev
                0x00000000000019e8        0xe /opt/ti/ccsv7/tools/compiler/gcc-arm-none-eabi-6-2017-q1-update/bin/../lib/gcc/arm-none-eabi/6.3.1/../../../../arm-none-eabi/lib/thumb/v7e-m/fpv4-sp/hard/libstdc++_nano.a(tinfo.o)
                0x00000000000019e8                std::type_info::~type_info()
 .text._ZNKSt9type_infoeqERKS_
                0x00000000000019f6       0x2c /opt/ti/ccsv7/tools/compiler/gcc-arm-none-eabi-6-2017-q1-update/bin/../lib/gcc/arm-none-eabi/6.3.1/../../../../arm-none-eabi/lib/thumb/v7e-m/fpv4-sp/hard/libstdc++_nano.a(tinfo.o)
                0x00000000000019f6                std::type_info::operator==(std::type_info const&) const
 .text._ZNKSt9type_info10__do_catchEPKS_PPvj
                0x0000000000001a22        0x4 /opt/ti/ccsv7/tools/compiler/gcc-arm-none-eabi-6-2017-q1-update/bin/../lib/gcc/arm-none-eabi/6.3.1/../../../../arm-none-eabi/lib/thumb/v7e-m/fpv4-sp/hard/libstdc++_nano.a(tinfo.o)
                0x0000000000001a22                std::type_info::__do_catch(std::type_info const*, void**, unsigned int) const
 .text._ZN10__cxxabiv111__terminateEPFvvE
                0x0000000000001a26        0x8 /opt/ti/ccsv7/tools/compiler/gcc-arm-none-eabi-6-2017-q1-update/bin/../lib/gcc/arm-none-eabi/6.3.1/../../../../arm-none-eabi/lib/thumb/v7e-m/fpv4-sp/hard/libstdc++_nano.a(eh_terminate.o)
                0x0000000000001a26                __cxxabiv1::__terminate(void (*)())
 *fill*         0x0000000000001a2e        0x2 
 .text._ZSt13set_terminatePFvvE
                0x0000000000001a30       0x20 /opt/ti/ccsv7/tools/compiler/gcc-arm-none-eabi-6-2017-q1-update/bin/../lib/gcc/arm-none-eabi/6.3.1/../../../../arm-none-eabi/lib/thumb/v7e-m/fpv4-sp/hard/libstdc++_nano.a(eh_terminate.o)
                0x0000000000001a30                std::set_terminate(void (*)())
 .text._ZSt13get_terminatev
                0x0000000000001a50       0x10 /opt/ti/ccsv7/tools/compiler/gcc-arm-none-eabi-6-2017-q1-update/bin/../lib/gcc/arm-none-eabi/6.3.1/../../../../arm-none-eabi/lib/thumb/v7e-m/fpv4-sp/hard/libstdc++_nano.a(eh_terminate.o)
                0x0000000000001a50                std::get_terminate()
 .text._ZSt9terminatev
                0x0000000000001a60        0xa /opt/ti/ccsv7/tools/compiler/gcc-arm-none-eabi-6-2017-q1-update/bin/../lib/gcc/arm-none-eabi/6.3.1/../../../../arm-none-eabi/lib/thumb/v7e-m/fpv4-sp/hard/libstdc++_nano.a(eh_terminate.o)
                0x0000000000001a60                std::terminate()
 .text._ZN10__cxxabiv112__unexpectedEPFvvE
                0x0000000000001a6a        0x8 /opt/ti/ccsv7/tools/compiler/gcc-arm-none-eabi-6-2017-q1-update/bin/../lib/gcc/arm-none-eabi/6.3.1/../../../../arm-none-eabi/lib/thumb/v7e-m/fpv4-sp/hard/libstdc++_nano.a(eh_terminate.o)
                0x0000000000001a6a                __cxxabiv1::__unexpected(void (*)())
 *fill*         0x0000000000001a72        0x2 
 .text._ZSt14set_unexpectedPFvvE
                0x0000000000001a74       0x20 /opt/ti/ccsv7/tools/compiler/gcc-arm-none-eabi-6-2017-q1-update/bin/../lib/gcc/arm-none-eabi/6.3.1/../../../../arm-none-eabi/lib/thumb/v7e-m/fpv4-sp/hard/libstdc++_nano.a(eh_terminate.o)
                0x0000000000001a74                std::set_unexpected(void (*)())
 .text._ZSt14get_unexpectedv
                0x0000000000001a94       0x10 /opt/ti/ccsv7/tools/compiler/gcc-arm-none-eabi-6-2017-q1-update/bin/../lib/gcc/arm-none-eabi/6.3.1/../../../../arm-none-eabi/lib/thumb/v7e-m/fpv4-sp/hard/libstdc++_nano.a(eh_terminate.o)
                0x0000000000001a94                std::get_unexpected()
 .text._ZSt10unexpectedv
                0x0000000000001aa4        0xa /opt/ti/ccsv7/tools/compiler/gcc-arm-none-eabi-6-2017-q1-update/bin/../lib/gcc/arm-none-eabi/6.3.1/../../../../arm-none-eabi/lib/thumb/v7e-m/fpv4-sp/hard/libstdc++_nano.a(eh_terminate.o)
                0x0000000000001aa4                std::unexpected()
 .text.abort    0x0000000000001aae        0xe /opt/ti/ccsv7/tools/compiler/gcc-arm-none-eabi-6-2017-q1-update/bin/../lib/gcc/arm-none-eabi/6.3.1/../../../../arm-none-eabi/lib/thumb/v7e-m/fpv4-sp/hard/libc_nano.a(lib_a-abort.o)
                0x0000000000001aae                abort
 .text.__cxa_atexit
                0x0000000000001abc       0x1c /opt/ti/ccsv7/tools/compiler/gcc-arm-none-eabi-6-2017-q1-update/bin/../lib/gcc/arm-none-eabi/6.3.1/../../../../arm-none-eabi/lib/thumb/v7e-m/fpv4-sp/hard/libc_nano.a(lib_a-cxa_atexit.o)
                0x0000000000001abc                __cxa_atexit
 .text.malloc   0x0000000000001ad8       0x10 /opt/ti/ccsv7/tools/compiler/gcc-arm-none-eabi-6-2017-q1-update/bin/../lib/gcc/arm-none-eabi/6.3.1/../../../../arm-none-eabi/lib/thumb/v7e-m/fpv4-sp/hard/libc_nano.a(lib_a-malloc.o)
                0x0000000000001ad8                malloc
 .text.free     0x0000000000001ae8       0x10 /opt/ti/ccsv7/tools/compiler/gcc-arm-none-eabi-6-2017-q1-update/bin/../lib/gcc/arm-none-eabi/6.3.1/../../../../arm-none-eabi/lib/thumb/v7e-m/fpv4-sp/hard/libc_nano.a(lib_a-malloc.o)
                0x0000000000001ae8                free
 .text._free_r  0x0000000000001af8       0x9c /opt/ti/ccsv7/tools/compiler/gcc-arm-none-eabi-6-2017-q1-update/bin/../lib/gcc/arm-none-eabi/6.3.1/../../../../arm-none-eabi/lib/thumb/v7e-m/fpv4-sp/hard/libc_nano.a(lib_a-nano-freer.o)
                0x0000000000001af8                _free_r
 .text._malloc_r
                0x0000000000001b94       0xbc /opt/ti/ccsv7/tools/compiler/gcc-arm-none-eabi-6-2017-q1-update/bin/../lib/gcc/arm-none-eabi/6.3.1/../../../../arm-none-eabi/lib/thumb/v7e-m/fpv4-sp/hard/libc_nano.a(lib_a-nano-mallocr.o)
                0x0000000000001b94                _malloc_r
 .text._sbrk_r  0x0000000000001c50       0x20 /opt/ti/ccsv7/tools/compiler/gcc-arm-none-eabi-6-2017-q1-update/bin/../lib/gcc/arm-none-eabi/6.3.1/../../../../arm-none-eabi/lib/thumb/v7e-m/fpv4-sp/hard/libc_nano.a(lib_a-sbrkr.o)
                0x0000000000001c50                _sbrk_r
 .text._init_signal_r
                0x0000000000001c70       0x2a /opt/ti/ccsv7/tools/compiler/gcc-arm-none-eabi-6-2017-q1-update/bin/../lib/gcc/arm-none-eabi/6.3.1/../../../../arm-none-eabi/lib/thumb/v7e-m/fpv4-sp/hard/libc_nano.a(lib_a-signal.o)
                0x0000000000001c70                _init_signal_r
 .text._signal_r
                0x0000000000001c9a       0x30 /opt/ti/ccsv7/tools/compiler/gcc-arm-none-eabi-6-2017-q1-update/bin/../lib/gcc/arm-none-eabi/6.3.1/../../../../arm-none-eabi/lib/thumb/v7e-m/fpv4-sp/hard/libc_nano.a(lib_a-signal.o)
                0x0000000000001c9a                _signal_r
 .text._raise_r
                0x0000000000001cca       0x50 /opt/ti/ccsv7/tools/compiler/gcc-arm-none-eabi-6-2017-q1-update/bin/../lib/gcc/arm-none-eabi/6.3.1/../../../../arm-none-eabi/lib/thumb/v7e-m/fpv4-sp/hard/libc_nano.a(lib_a-signal.o)
                0x0000000000001cca                _raise_r
 .text.__sigtramp_r
                0x0000000000001d1a       0x48 /opt/ti/ccsv7/tools/compiler/gcc-arm-none-eabi-6-2017-q1-update/bin/../lib/gcc/arm-none-eabi/6.3.1/../../../../arm-none-eabi/lib/thumb/v7e-m/fpv4-sp/hard/libc_nano.a(lib_a-signal.o)
                0x0000000000001d1a                __sigtramp_r
 *fill*         0x0000000000001d62        0x2 
 .text.raise    0x0000000000001d64       0x10 /opt/ti/ccsv7/tools/compiler/gcc-arm-none-eabi-6-2017-q1-update/bin/../lib/gcc/arm-none-eabi/6.3.1/../../../../arm-none-eabi/lib/thumb/v7e-m/fpv4-sp/hard/libc_nano.a(lib_a-signal.o)
                0x0000000000001d64                raise
 .text.signal   0x0000000000001d74       0x10 /opt/ti/ccsv7/tools/compiler/gcc-arm-none-eabi-6-2017-q1-update/bin/../lib/gcc/arm-none-eabi/6.3.1/../../../../arm-none-eabi/lib/thumb/v7e-m/fpv4-sp/hard/libc_nano.a(lib_a-signal.o)
                0x0000000000001d74                signal
 .text._init_signal
                0x0000000000001d84        0xc /opt/ti/ccsv7/tools/compiler/gcc-arm-none-eabi-6-2017-q1-update/bin/../lib/gcc/arm-none-eabi/6.3.1/../../../../arm-none-eabi/lib/thumb/v7e-m/fpv4-sp/hard/libc_nano.a(lib_a-signal.o)
                0x0000000000001d84                _init_signal
 .text.__sigtramp
                0x0000000000001d90       0x10 /opt/ti/ccsv7/tools/compiler/gcc-arm-none-eabi-6-2017-q1-update/bin/../lib/gcc/arm-none-eabi/6.3.1/../../../../arm-none-eabi/lib/thumb/v7e-m/fpv4-sp/hard/libc_nano.a(lib_a-signal.o)
                0x0000000000001d90                __sigtramp
 .text._kill_r  0x0000000000001da0       0x24 /opt/ti/ccsv7/tools/compiler/gcc-arm-none-eabi-6-2017-q1-update/bin/../lib/gcc/arm-none-eabi/6.3.1/../../../../arm-none-eabi/lib/thumb/v7e-m/fpv4-sp/hard/libc_nano.a(lib_a-signalr.o)
                0x0000000000001da0                _kill_r
 .text._getpid_r
                0x0000000000001dc4        0x4 /opt/ti/ccsv7/tools/compiler/gcc-arm-none-eabi-6-2017-q1-update/bin/../lib/gcc/arm-none-eabi/6.3.1/../../../../arm-none-eabi/lib/thumb/v7e-m/fpv4-sp/hard/libc_nano.a(lib_a-signalr.o)
                0x0000000000001dc4                _getpid_r
 .text.__malloc_lock
                0x0000000000001dc8        0x2 /opt/ti/ccsv7/tools/compiler/gcc-arm-none-eabi-6-2017-q1-update/bin/../lib/gcc/arm-none-eabi/6.3.1/../../../../arm-none-eabi/lib/thumb/v7e-m/fpv4-sp/hard/libc_nano.a(lib_a-mlock.o)
                0x0000000000001dc8                __malloc_lock
 .text.__malloc_unlock
                0x0000000000001dca        0x2 /opt/ti/ccsv7/tools/compiler/gcc-arm-none-eabi-6-2017-q1-update/bin/../lib/gcc/arm-none-eabi/6.3.1/../../../../arm-none-eabi/lib/thumb/v7e-m/fpv4-sp/hard/libc_nano.a(lib_a-mlock.o)
                0x0000000000001dca                __malloc_unlock
 .text.cleanup_glue
                0x0000000000001dcc       0x1a /opt/ti/ccsv7/tools/compiler/gcc-arm-none-eabi-6-2017-q1-update/bin/../lib/gcc/arm-none-eabi/6.3.1/../../../../arm-none-eabi/lib/thumb/v7e-m/fpv4-sp/hard/libc_nano.a(lib_a-reent.o)
                0x0000000000001dcc                cleanup_glue
 *fill*         0x0000000000001de6        0x2 
 .text._reclaim_reent
                0x0000000000001de8       0xb8 /opt/ti/ccsv7/tools/compiler/gcc-arm-none-eabi-6-2017-q1-update/bin/../lib/gcc/arm-none-eabi/6.3.1/../../../../arm-none-eabi/lib/thumb/v7e-m/fpv4-sp/hard/libc_nano.a(lib_a-reent.o)
                0x0000000000001de8                _reclaim_reent
 .text._getpid  0x0000000000001ea0       0x10 /opt/ti/ccsv7/tools/compiler/gcc-arm-none-eabi-6-2017-q1-update/bin/../lib/gcc/arm-none-eabi/6.3.1/../../../../arm-none-eabi/lib/thumb/v7e-m/fpv4-sp/hard/libnosys.a(getpid.o)
                0x0000000000001ea0                _getpid
 .text._kill    0x0000000000001eb0       0x10 /opt/ti/ccsv7/tools/compiler/gcc-arm-none-eabi-6-2017-q1-update/bin/../lib/gcc/arm-none-eabi/6.3.1/../../../../arm-none-eabi/lib/thumb/v7e-m/fpv4-sp/hard/libnosys.a(kill.o)
                0x0000000000001eb0                _kill
 .text._sbrk    0x0000000000001ec0       0x1c /opt/ti/ccsv7/tools/compiler/gcc-arm-none-eabi-6-2017-q1-update/bin/../lib/gcc/arm-none-eabi/6.3.1/../../../../arm-none-eabi/lib/thumb/v7e-m/fpv4-sp/hard/libnosys.a(sbrk.o)
                0x0000000000001ec0                _sbrk
                0x0000000000001edc                . = ALIGN (0x4)
 *(.ctors)
                0x0000000000001edc                . = ALIGN (0x4)
 *(.dtors)
                0x0000000000001edc                . = ALIGN (0x4)
                0x0000000000001edc                __init_array_start = .
 *(.init_array*)
 .init_array    0x0000000000001edc        0x4 /opt/ti/ccsv7/tools/compiler/gcc-arm-none-eabi-6-2017-q1-update/bin/../lib/gcc/arm-none-eabi/6.3.1/thumb/v7e-m/fpv4-sp/hard/crtbegin.o
 .init_array    0x0000000000001ee0        0x4 /home/student/git/workspace_mct/YAHAL/libYAHAL_msp432.a(gpio_msp432.cpp.o)
                0x0000000000001ee4                __init_array_end = .
 *(.init)
 .init          0x0000000000001ee4        0x4 /opt/ti/ccsv7/tools/compiler/gcc-arm-none-eabi-6-2017-q1-update/bin/../lib/gcc/arm-none-eabi/6.3.1/thumb/v7e-m/fpv4-sp/hard/crti.o
                0x0000000000001ee4                _init
 .init          0x0000000000001ee8        0x8 /opt/ti/ccsv7/tools/compiler/gcc-arm-none-eabi-6-2017-q1-update/bin/../lib/gcc/arm-none-eabi/6.3.1/thumb/v7e-m/fpv4-sp/hard/crtn.o
 *(.fini*)
 .fini          0x0000000000001ef0        0x4 /opt/ti/ccsv7/tools/compiler/gcc-arm-none-eabi-6-2017-q1-update/bin/../lib/gcc/arm-none-eabi/6.3.1/thumb/v7e-m/fpv4-sp/hard/crti.o
                0x0000000000001ef0                _fini
 .fini_array    0x0000000000001ef4        0x4 /opt/ti/ccsv7/tools/compiler/gcc-arm-none-eabi-6-2017-q1-update/bin/../lib/gcc/arm-none-eabi/6.3.1/thumb/v7e-m/fpv4-sp/hard/crtbegin.o
 .fini          0x0000000000001ef8        0x8 /opt/ti/ccsv7/tools/compiler/gcc-arm-none-eabi-6-2017-q1-update/bin/../lib/gcc/arm-none-eabi/6.3.1/thumb/v7e-m/fpv4-sp/hard/crtn.o

.glue_7         0x0000000000001f00        0x0
 .glue_7        0x0000000000001f00        0x0 linker stubs

.glue_7t        0x0000000000001f00        0x0
 .glue_7t       0x0000000000001f00        0x0 linker stubs

.vfp11_veneer   0x0000000000001f00        0x0
 .vfp11_veneer  0x0000000000001f00        0x0 linker stubs

.v4_bx          0x0000000000001f00        0x0
 .v4_bx         0x0000000000001f00        0x0 linker stubs

.iplt           0x0000000000001f00        0x0
 .iplt          0x0000000000001f00        0x0 /opt/ti/ccsv7/tools/compiler/gcc-arm-none-eabi-6-2017-q1-update/bin/../lib/gcc/arm-none-eabi/6.3.1/thumb/v7e-m/fpv4-sp/hard/crtbegin.o

.rodata         0x0000000000001f00      0x28c
 *(.rodata)
 .rodata        0x0000000000001f00       0x24 /home/student/git/workspace_mct/YAHAL/libYAHAL_msp432.a(gpio_msp432.cpp.o)
 *(.rodata.*)
 .rodata._global_impure_ptr
                0x0000000000001f24        0x4 /opt/ti/ccsv7/tools/compiler/gcc-arm-none-eabi-6-2017-q1-update/bin/../lib/gcc/arm-none-eabi/6.3.1/../../../../arm-none-eabi/lib/thumb/v7e-m/fpv4-sp/hard/libc_nano.a(lib_a-impure.o)
                0x0000000000001f24                _global_impure_ptr
 .rodata._ZN4GPIOL5INPUTE
                0x0000000000001f28        0x2 Debug/main.cpp.o
 .rodata._ZN4GPIOL6OUTPUTE
                0x0000000000001f2a        0x2 Debug/main.cpp.o
 .rodata._ZN4GPIOL17OUTPUT_OPEN_DRAINE
                0x0000000000001f2c        0x2 Debug/main.cpp.o
 .rodata._ZN4GPIOL18OUTPUT_OPEN_SOURCEE
                0x0000000000001f2e        0x2 Debug/main.cpp.o
 .rodata._ZN4GPIOL6PULLUPE
                0x0000000000001f30        0x2 Debug/main.cpp.o
 .rodata._ZN4GPIOL8PULLDOWNE
                0x0000000000001f32        0x2 Debug/main.cpp.o
 .rodata._ZN4GPIOL4SLOWE
                0x0000000000001f34        0x2 Debug/main.cpp.o
 .rodata._ZN4GPIOL4FASTE
                0x0000000000001f36        0x2 Debug/main.cpp.o
 .rodata._ZN4GPIOL9INIT_HIGHE
                0x0000000000001f38        0x2 Debug/main.cpp.o
 .rodata._ZN4GPIOL8INIT_LOWE
                0x0000000000001f3a        0x2 Debug/main.cpp.o
 .rodata._ZN4GPIOL6RISINGE
                0x0000000000001f3c        0x2 Debug/main.cpp.o
 .rodata._ZN4GPIOL7FALLINGE
                0x0000000000001f3e        0x2 Debug/main.cpp.o
 .rodata._ZN4GPIOL10LEVEL_HIGHE
                0x0000000000001f40        0x2 Debug/main.cpp.o
 .rodata._ZN4GPIOL9LEVEL_LOWE
                0x0000000000001f42        0x2 Debug/main.cpp.o
 .rodata._ZN4GPIOL5INPUTE
                0x0000000000001f44        0x2 /home/student/git/workspace_mct/YAHAL/libYAHAL_msp432.a(gpio_msp432.cpp.o)
 .rodata._ZN4GPIOL6OUTPUTE
                0x0000000000001f46        0x2 /home/student/git/workspace_mct/YAHAL/libYAHAL_msp432.a(gpio_msp432.cpp.o)
 .rodata._ZN4GPIOL17OUTPUT_OPEN_DRAINE
                0x0000000000001f48        0x2 /home/student/git/workspace_mct/YAHAL/libYAHAL_msp432.a(gpio_msp432.cpp.o)
 .rodata._ZN4GPIOL18OUTPUT_OPEN_SOURCEE
                0x0000000000001f4a        0x2 /home/student/git/workspace_mct/YAHAL/libYAHAL_msp432.a(gpio_msp432.cpp.o)
 .rodata._ZN4GPIOL6PULLUPE
                0x0000000000001f4c        0x2 /home/student/git/workspace_mct/YAHAL/libYAHAL_msp432.a(gpio_msp432.cpp.o)
 .rodata._ZN4GPIOL8PULLDOWNE
                0x0000000000001f4e        0x2 /home/student/git/workspace_mct/YAHAL/libYAHAL_msp432.a(gpio_msp432.cpp.o)
 .rodata._ZN4GPIOL4SLOWE
                0x0000000000001f50        0x2 /home/student/git/workspace_mct/YAHAL/libYAHAL_msp432.a(gpio_msp432.cpp.o)
 .rodata._ZN4GPIOL4FASTE
                0x0000000000001f52        0x2 /home/student/git/workspace_mct/YAHAL/libYAHAL_msp432.a(gpio_msp432.cpp.o)
 .rodata._ZN4GPIOL9INIT_HIGHE
                0x0000000000001f54        0x2 /home/student/git/workspace_mct/YAHAL/libYAHAL_msp432.a(gpio_msp432.cpp.o)
 .rodata._ZN4GPIOL8INIT_LOWE
                0x0000000000001f56        0x2 /home/student/git/workspace_mct/YAHAL/libYAHAL_msp432.a(gpio_msp432.cpp.o)
 .rodata._ZN4GPIOL6RISINGE
                0x0000000000001f58        0x2 /home/student/git/workspace_mct/YAHAL/libYAHAL_msp432.a(gpio_msp432.cpp.o)
 .rodata._ZN4GPIOL7FALLINGE
                0x0000000000001f5a        0x2 /home/student/git/workspace_mct/YAHAL/libYAHAL_msp432.a(gpio_msp432.cpp.o)
 .rodata._ZN4GPIOL10LEVEL_HIGHE
                0x0000000000001f5c        0x2 /home/student/git/workspace_mct/YAHAL/libYAHAL_msp432.a(gpio_msp432.cpp.o)
 .rodata._ZN4GPIOL9LEVEL_LOWE
                0x0000000000001f5e        0x2 /home/student/git/workspace_mct/YAHAL/libYAHAL_msp432.a(gpio_msp432.cpp.o)
 .rodata._ZTV11gpio_msp432
                0x0000000000001f60       0x30 /home/student/git/workspace_mct/YAHAL/libYAHAL_msp432.a(gpio_msp432.cpp.o)
                0x0000000000001f60                vtable for gpio_msp432
 .rodata._ZTV14gpio_interface
                0x0000000000001f90       0x30 /home/student/git/workspace_mct/YAHAL/libYAHAL_msp432.a(gpio_msp432.cpp.o)
                0x0000000000001f90                vtable for gpio_interface
 .rodata._ZTI11gpio_msp432
                0x0000000000001fc0        0xc /home/student/git/workspace_mct/YAHAL/libYAHAL_msp432.a(gpio_msp432.cpp.o)
                0x0000000000001fc0                typeinfo for gpio_msp432
 .rodata._ZTS11gpio_msp432
                0x0000000000001fcc        0xe /home/student/git/workspace_mct/YAHAL/libYAHAL_msp432.a(gpio_msp432.cpp.o)
                0x0000000000001fcc                typeinfo name for gpio_msp432
 *fill*         0x0000000000001fda        0x2 
 .rodata._ZTI14gpio_interface
                0x0000000000001fdc        0x8 /home/student/git/workspace_mct/YAHAL/libYAHAL_msp432.a(gpio_msp432.cpp.o)
                0x0000000000001fdc                typeinfo for gpio_interface
 .rodata._ZTS14gpio_interface
                0x0000000000001fe4       0x11 /home/student/git/workspace_mct/YAHAL/libYAHAL_msp432.a(gpio_msp432.cpp.o)
                0x0000000000001fe4                typeinfo name for gpio_interface
 *fill*         0x0000000000001ff5        0x3 
 .rodata._ZTV12timer_msp432
                0x0000000000001ff8       0x30 /home/student/git/workspace_mct/YAHAL/libYAHAL_msp432.a(timer_msp432.cpp.o)
                0x0000000000001ff8                vtable for timer_msp432
 .rodata._ZTV15timer_interface
                0x0000000000002028       0x30 /home/student/git/workspace_mct/YAHAL/libYAHAL_msp432.a(timer_msp432.cpp.o)
                0x0000000000002028                vtable for timer_interface
 .rodata._ZTI12timer_msp432
                0x0000000000002058        0xc /home/student/git/workspace_mct/YAHAL/libYAHAL_msp432.a(timer_msp432.cpp.o)
                0x0000000000002058                typeinfo for timer_msp432
 .rodata._ZTS12timer_msp432
                0x0000000000002064        0xf /home/student/git/workspace_mct/YAHAL/libYAHAL_msp432.a(timer_msp432.cpp.o)
                0x0000000000002064                typeinfo name for timer_msp432
 *fill*         0x0000000000002073        0x1 
 .rodata._ZTI15timer_interface
                0x0000000000002074        0x8 /home/student/git/workspace_mct/YAHAL/libYAHAL_msp432.a(timer_msp432.cpp.o)
                0x0000000000002074                typeinfo for timer_interface
 .rodata._ZTS15timer_interface
                0x000000000000207c       0x12 /home/student/git/workspace_mct/YAHAL/libYAHAL_msp432.a(timer_msp432.cpp.o)
                0x000000000000207c                typeinfo name for timer_interface
 *fill*         0x000000000000208e        0x2 
 .rodata._ZTIN10__cxxabiv117__class_type_infoE
                0x0000000000002090        0xc /opt/ti/ccsv7/tools/compiler/gcc-arm-none-eabi-6-2017-q1-update/bin/../lib/gcc/arm-none-eabi/6.3.1/../../../../arm-none-eabi/lib/thumb/v7e-m/fpv4-sp/hard/libstdc++_nano.a(class_type_info.o)
                0x0000000000002090                typeinfo for __cxxabiv1::__class_type_info
 .rodata._ZTSN10__cxxabiv117__class_type_infoE
                0x000000000000209c       0x22 /opt/ti/ccsv7/tools/compiler/gcc-arm-none-eabi-6-2017-q1-update/bin/../lib/gcc/arm-none-eabi/6.3.1/../../../../arm-none-eabi/lib/thumb/v7e-m/fpv4-sp/hard/libstdc++_nano.a(class_type_info.o)
                0x000000000000209c                typeinfo name for __cxxabiv1::__class_type_info
 *fill*         0x00000000000020be        0x2 
 .rodata._ZTVN10__cxxabiv117__class_type_infoE
                0x00000000000020c0       0x2c /opt/ti/ccsv7/tools/compiler/gcc-arm-none-eabi-6-2017-q1-update/bin/../lib/gcc/arm-none-eabi/6.3.1/../../../../arm-none-eabi/lib/thumb/v7e-m/fpv4-sp/hard/libstdc++_nano.a(class_type_info.o)
                0x00000000000020c0                vtable for __cxxabiv1::__class_type_info
 .rodata._ZTIN10__cxxabiv120__si_class_type_infoE
                0x00000000000020ec        0xc /opt/ti/ccsv7/tools/compiler/gcc-arm-none-eabi-6-2017-q1-update/bin/../lib/gcc/arm-none-eabi/6.3.1/../../../../arm-none-eabi/lib/thumb/v7e-m/fpv4-sp/hard/libstdc++_nano.a(si_class_type_info.o)
                0x00000000000020ec                typeinfo for __cxxabiv1::__si_class_type_info
 .rodata._ZTSN10__cxxabiv120__si_class_type_infoE
                0x00000000000020f8       0x25 /opt/ti/ccsv7/tools/compiler/gcc-arm-none-eabi-6-2017-q1-update/bin/../lib/gcc/arm-none-eabi/6.3.1/../../../../arm-none-eabi/lib/thumb/v7e-m/fpv4-sp/hard/libstdc++_nano.a(si_class_type_info.o)
                0x00000000000020f8                typeinfo name for __cxxabiv1::__si_class_type_info
 *fill*         0x000000000000211d        0x3 
 .rodata._ZTVN10__cxxabiv120__si_class_type_infoE
                0x0000000000002120       0x2c /opt/ti/ccsv7/tools/compiler/gcc-arm-none-eabi-6-2017-q1-update/bin/../lib/gcc/arm-none-eabi/6.3.1/../../../../arm-none-eabi/lib/thumb/v7e-m/fpv4-sp/hard/libstdc++_nano.a(si_class_type_info.o)
                0x0000000000002120                vtable for __cxxabiv1::__si_class_type_info
 .rodata._ZTISt9type_info
                0x000000000000214c        0x8 /opt/ti/ccsv7/tools/compiler/gcc-arm-none-eabi-6-2017-q1-update/bin/../lib/gcc/arm-none-eabi/6.3.1/../../../../arm-none-eabi/lib/thumb/v7e-m/fpv4-sp/hard/libstdc++_nano.a(tinfo.o)
                0x000000000000214c                typeinfo for std::type_info
 .rodata._ZTSSt9type_info
                0x0000000000002154        0xd /opt/ti/ccsv7/tools/compiler/gcc-arm-none-eabi-6-2017-q1-update/bin/../lib/gcc/arm-none-eabi/6.3.1/../../../../arm-none-eabi/lib/thumb/v7e-m/fpv4-sp/hard/libstdc++_nano.a(tinfo.o)
                0x0000000000002154                typeinfo name for std::type_info
 *fill*         0x0000000000002161        0x3 
 .rodata._ZTVSt9type_info
                0x0000000000002164       0x20 /opt/ti/ccsv7/tools/compiler/gcc-arm-none-eabi-6-2017-q1-update/bin/../lib/gcc/arm-none-eabi/6.3.1/../../../../arm-none-eabi/lib/thumb/v7e-m/fpv4-sp/hard/libstdc++_nano.a(tinfo.o)
                0x0000000000002164                vtable for std::type_info
 .rodata.__cxa_atexit_dummy
                0x0000000000002184        0x4 /opt/ti/ccsv7/tools/compiler/gcc-arm-none-eabi-6-2017-q1-update/bin/../lib/gcc/arm-none-eabi/6.3.1/../../../../arm-none-eabi/lib/thumb/v7e-m/fpv4-sp/hard/libc_nano.a(lib_a-cxa_atexit.o)
                0x0000000000002184                __cxa_atexit_dummy
 .rodata.__on_exit_args
                0x0000000000002188        0x4 /opt/ti/ccsv7/tools/compiler/gcc-arm-none-eabi-6-2017-q1-update/bin/../lib/gcc/arm-none-eabi/6.3.1/../../../../arm-none-eabi/lib/thumb/v7e-m/fpv4-sp/hard/libc_nano.a(lib_a-on_exit_args.o)
                0x0000000000002188                __on_exit_args

.eh_frame       0x000000000000218c        0x4
 .eh_frame      0x000000000000218c        0x0 /opt/ti/ccsv7/tools/compiler/gcc-arm-none-eabi-6-2017-q1-update/bin/../lib/gcc/arm-none-eabi/6.3.1/thumb/v7e-m/fpv4-sp/hard/crtbegin.o
 .eh_frame      0x000000000000218c        0x4 /opt/ti/ccsv7/tools/compiler/gcc-arm-none-eabi-6-2017-q1-update/bin/../lib/gcc/arm-none-eabi/6.3.1/thumb/v7e-m/fpv4-sp/hard/crtend.o

.ARM.exidx      0x0000000000002190        0x8
                0x0000000000002190                __exidx_start = .
 *(.ARM.exidx* .gnu.linkonce.armexidx.*)
 .ARM.exidx     0x0000000000002190        0x8 /opt/ti/ccsv7/tools/compiler/gcc-arm-none-eabi-6-2017-q1-update/bin/../lib/gcc/arm-none-eabi/6.3.1/../../../../arm-none-eabi/lib/thumb/v7e-m/fpv4-sp/hard/crt0.o
                0x0000000000002198                __exidx_end = .

.ARM.extab      0x0000000000002198        0x0
 *(.ARM.extab* .gnu.linkonce.armextab.*)
 .ARM.extab     0x0000000000002198        0x0 /opt/ti/ccsv7/tools/compiler/gcc-arm-none-eabi-6-2017-q1-update/bin/../lib/gcc/arm-none-eabi/6.3.1/../../../../arm-none-eabi/lib/thumb/v7e-m/fpv4-sp/hard/crt0.o
                0x0000000000002198                __etext = .

.rel.dyn        0x0000000000002198        0x0
 .rel.iplt      0x0000000000002198        0x0 /opt/ti/ccsv7/tools/compiler/gcc-arm-none-eabi-6-2017-q1-update/bin/../lib/gcc/arm-none-eabi/6.3.1/thumb/v7e-m/fpv4-sp/hard/crtbegin.o

.data           0x0000000020000000       0x9c load address 0x0000000000002198
                0x0000000000002198                __data_load__ = LOADADDR (.data)
                0x0000000020000000                __data_start__ = .
 *(.data)
 .data          0x0000000020000000        0x0 /opt/ti/ccsv7/tools/compiler/gcc-arm-none-eabi-6-2017-q1-update/bin/../lib/gcc/arm-none-eabi/6.3.1/thumb/v7e-m/fpv4-sp/hard/crti.o
 .data          0x0000000020000000        0x4 /opt/ti/ccsv7/tools/compiler/gcc-arm-none-eabi-6-2017-q1-update/bin/../lib/gcc/arm-none-eabi/6.3.1/thumb/v7e-m/fpv4-sp/hard/crtbegin.o
                0x0000000020000000                __dso_handle
 .data          0x0000000020000004        0x0 /opt/ti/ccsv7/tools/compiler/gcc-arm-none-eabi-6-2017-q1-update/bin/../lib/gcc/arm-none-eabi/6.3.1/../../../../arm-none-eabi/lib/thumb/v7e-m/fpv4-sp/hard/crt0.o
 .data          0x0000000020000004        0x0 /opt/ti/ccsv7/tools/compiler/gcc-arm-none-eabi-6-2017-q1-update/bin/../lib/gcc/arm-none-eabi/6.3.1/../../../../arm-none-eabi/lib/thumb/v7e-m/fpv4-sp/hard/libc_nano.a(lib_a-exit.o)
 .data          0x0000000020000004        0x0 /opt/ti/ccsv7/tools/compiler/gcc-arm-none-eabi-6-2017-q1-update/bin/../lib/gcc/arm-none-eabi/6.3.1/../../../../arm-none-eabi/lib/thumb/v7e-m/fpv4-sp/hard/libc_nano.a(lib_a-impure.o)
 .data          0x0000000020000004        0x0 /opt/ti/ccsv7/tools/compiler/gcc-arm-none-eabi-6-2017-q1-update/bin/../lib/gcc/arm-none-eabi/6.3.1/../../../../arm-none-eabi/lib/thumb/v7e-m/fpv4-sp/hard/libc_nano.a(lib_a-init.o)
 .data          0x0000000020000004        0x0 /opt/ti/ccsv7/tools/compiler/gcc-arm-none-eabi-6-2017-q1-update/bin/../lib/gcc/arm-none-eabi/6.3.1/../../../../arm-none-eabi/lib/thumb/v7e-m/fpv4-sp/hard/libc_nano.a(lib_a-memset.o)
 .data          0x0000000020000004        0x0 /opt/ti/ccsv7/tools/compiler/gcc-arm-none-eabi-6-2017-q1-update/bin/../lib/gcc/arm-none-eabi/6.3.1/../../../../arm-none-eabi/lib/thumb/v7e-m/fpv4-sp/hard/libnosys.a(_exit.o)
 .data          0x0000000020000004        0x0 Debug/main.cpp.o
 .data          0x0000000020000004        0x0 Debug/startup_msp432p401r_gcc.c.o
 .data          0x0000000020000004        0x0 Debug/system_msp432p401r.c.o
 .data          0x0000000020000004        0x0 /home/student/git/workspace_mct/YAHAL/libYAHAL_msp432.a(gpio_msp432.cpp.o)
 .data          0x0000000020000004        0x0 /home/student/git/workspace_mct/YAHAL/libYAHAL_msp432.a(timer_msp432.cpp.o)
 .data          0x0000000020000004        0x0 /opt/ti/ccsv7/tools/compiler/gcc-arm-none-eabi-6-2017-q1-update/bin/../lib/gcc/arm-none-eabi/6.3.1/../../../../arm-none-eabi/lib/thumb/v7e-m/fpv4-sp/hard/libstdc++_nano.a(class_type_info.o)
 .data          0x0000000020000004        0x0 /opt/ti/ccsv7/tools/compiler/gcc-arm-none-eabi-6-2017-q1-update/bin/../lib/gcc/arm-none-eabi/6.3.1/../../../../arm-none-eabi/lib/thumb/v7e-m/fpv4-sp/hard/libstdc++_nano.a(atexit_arm.o)
 .data          0x0000000020000004        0x0 /opt/ti/ccsv7/tools/compiler/gcc-arm-none-eabi-6-2017-q1-update/bin/../lib/gcc/arm-none-eabi/6.3.1/../../../../arm-none-eabi/lib/thumb/v7e-m/fpv4-sp/hard/libstdc++_nano.a(si_class_type_info.o)
 .data          0x0000000020000004        0x0 /opt/ti/ccsv7/tools/compiler/gcc-arm-none-eabi-6-2017-q1-update/bin/../lib/gcc/arm-none-eabi/6.3.1/../../../../arm-none-eabi/lib/thumb/v7e-m/fpv4-sp/hard/libstdc++_nano.a(del_ops.o)
 .data          0x0000000020000004        0x0 /opt/ti/ccsv7/tools/compiler/gcc-arm-none-eabi-6-2017-q1-update/bin/../lib/gcc/arm-none-eabi/6.3.1/../../../../arm-none-eabi/lib/thumb/v7e-m/fpv4-sp/hard/libstdc++_nano.a(del_op.o)
 .data          0x0000000020000004        0x0 /opt/ti/ccsv7/tools/compiler/gcc-arm-none-eabi-6-2017-q1-update/bin/../lib/gcc/arm-none-eabi/6.3.1/../../../../arm-none-eabi/lib/thumb/v7e-m/fpv4-sp/hard/libstdc++_nano.a(pure.o)
 .data          0x0000000020000004        0x0 /opt/ti/ccsv7/tools/compiler/gcc-arm-none-eabi-6-2017-q1-update/bin/../lib/gcc/arm-none-eabi/6.3.1/../../../../arm-none-eabi/lib/thumb/v7e-m/fpv4-sp/hard/libstdc++_nano.a(tinfo.o)
 .data          0x0000000020000004        0x0 /opt/ti/ccsv7/tools/compiler/gcc-arm-none-eabi-6-2017-q1-update/bin/../lib/gcc/arm-none-eabi/6.3.1/../../../../arm-none-eabi/lib/thumb/v7e-m/fpv4-sp/hard/libstdc++_nano.a(eh_terminate.o)
 .data          0x0000000020000004        0x0 /opt/ti/ccsv7/tools/compiler/gcc-arm-none-eabi-6-2017-q1-update/bin/../lib/gcc/arm-none-eabi/6.3.1/../../../../arm-none-eabi/lib/thumb/v7e-m/fpv4-sp/hard/libstdc++_nano.a(eh_term_handler.o)
 .data          0x0000000020000004        0x0 /opt/ti/ccsv7/tools/compiler/gcc-arm-none-eabi-6-2017-q1-update/bin/../lib/gcc/arm-none-eabi/6.3.1/../../../../arm-none-eabi/lib/thumb/v7e-m/fpv4-sp/hard/libstdc++_nano.a(eh_unex_handler.o)
 .data          0x0000000020000004        0x0 /opt/ti/ccsv7/tools/compiler/gcc-arm-none-eabi-6-2017-q1-update/bin/../lib/gcc/arm-none-eabi/6.3.1/../../../../arm-none-eabi/lib/thumb/v7e-m/fpv4-sp/hard/libc_nano.a(lib_a-abort.o)
 .data          0x0000000020000004        0x0 /opt/ti/ccsv7/tools/compiler/gcc-arm-none-eabi-6-2017-q1-update/bin/../lib/gcc/arm-none-eabi/6.3.1/../../../../arm-none-eabi/lib/thumb/v7e-m/fpv4-sp/hard/libc_nano.a(lib_a-cxa_atexit.o)
 .data          0x0000000020000004        0x0 /opt/ti/ccsv7/tools/compiler/gcc-arm-none-eabi-6-2017-q1-update/bin/../lib/gcc/arm-none-eabi/6.3.1/../../../../arm-none-eabi/lib/thumb/v7e-m/fpv4-sp/hard/libc_nano.a(lib_a-malloc.o)
 .data          0x0000000020000004        0x0 /opt/ti/ccsv7/tools/compiler/gcc-arm-none-eabi-6-2017-q1-update/bin/../lib/gcc/arm-none-eabi/6.3.1/../../../../arm-none-eabi/lib/thumb/v7e-m/fpv4-sp/hard/libc_nano.a(lib_a-nano-freer.o)
 .data          0x0000000020000004        0x0 /opt/ti/ccsv7/tools/compiler/gcc-arm-none-eabi-6-2017-q1-update/bin/../lib/gcc/arm-none-eabi/6.3.1/../../../../arm-none-eabi/lib/thumb/v7e-m/fpv4-sp/hard/libc_nano.a(lib_a-nano-mallocr.o)
 .data          0x0000000020000004        0x0 /opt/ti/ccsv7/tools/compiler/gcc-arm-none-eabi-6-2017-q1-update/bin/../lib/gcc/arm-none-eabi/6.3.1/../../../../arm-none-eabi/lib/thumb/v7e-m/fpv4-sp/hard/libc_nano.a(lib_a-on_exit_args.o)
 .data          0x0000000020000004        0x0 /opt/ti/ccsv7/tools/compiler/gcc-arm-none-eabi-6-2017-q1-update/bin/../lib/gcc/arm-none-eabi/6.3.1/../../../../arm-none-eabi/lib/thumb/v7e-m/fpv4-sp/hard/libc_nano.a(lib_a-sbrkr.o)
 .data          0x0000000020000004        0x0 /opt/ti/ccsv7/tools/compiler/gcc-arm-none-eabi-6-2017-q1-update/bin/../lib/gcc/arm-none-eabi/6.3.1/../../../../arm-none-eabi/lib/thumb/v7e-m/fpv4-sp/hard/libc_nano.a(lib_a-signal.o)
 .data          0x0000000020000004        0x0 /opt/ti/ccsv7/tools/compiler/gcc-arm-none-eabi-6-2017-q1-update/bin/../lib/gcc/arm-none-eabi/6.3.1/../../../../arm-none-eabi/lib/thumb/v7e-m/fpv4-sp/hard/libc_nano.a(lib_a-signalr.o)
 .data          0x0000000020000004        0x0 /opt/ti/ccsv7/tools/compiler/gcc-arm-none-eabi-6-2017-q1-update/bin/../lib/gcc/arm-none-eabi/6.3.1/../../../../arm-none-eabi/lib/thumb/v7e-m/fpv4-sp/hard/libc_nano.a(lib_a-strcmp.o)
 .data          0x0000000020000004        0x0 /opt/ti/ccsv7/tools/compiler/gcc-arm-none-eabi-6-2017-q1-update/bin/../lib/gcc/arm-none-eabi/6.3.1/../../../../arm-none-eabi/lib/thumb/v7e-m/fpv4-sp/hard/libc_nano.a(lib_a-mlock.o)
 .data          0x0000000020000004        0x0 /opt/ti/ccsv7/tools/compiler/gcc-arm-none-eabi-6-2017-q1-update/bin/../lib/gcc/arm-none-eabi/6.3.1/../../../../arm-none-eabi/lib/thumb/v7e-m/fpv4-sp/hard/libc_nano.a(lib_a-reent.o)
 .data          0x0000000020000004        0x0 /opt/ti/ccsv7/tools/compiler/gcc-arm-none-eabi-6-2017-q1-update/bin/../lib/gcc/arm-none-eabi/6.3.1/../../../../arm-none-eabi/lib/thumb/v7e-m/fpv4-sp/hard/libnosys.a(getpid.o)
 .data          0x0000000020000004        0x0 /opt/ti/ccsv7/tools/compiler/gcc-arm-none-eabi-6-2017-q1-update/bin/../lib/gcc/arm-none-eabi/6.3.1/../../../../arm-none-eabi/lib/thumb/v7e-m/fpv4-sp/hard/libnosys.a(kill.o)
 .data          0x0000000020000004        0x0 /opt/ti/ccsv7/tools/compiler/gcc-arm-none-eabi-6-2017-q1-update/bin/../lib/gcc/arm-none-eabi/6.3.1/../../../../arm-none-eabi/lib/thumb/v7e-m/fpv4-sp/hard/libnosys.a(sbrk.o)
 .data          0x0000000020000004        0x0 /opt/ti/ccsv7/tools/compiler/gcc-arm-none-eabi-6-2017-q1-update/bin/../lib/gcc/arm-none-eabi/6.3.1/thumb/v7e-m/fpv4-sp/hard/crtend.o
 .data          0x0000000020000004        0x0 /opt/ti/ccsv7/tools/compiler/gcc-arm-none-eabi-6-2017-q1-update/bin/../lib/gcc/arm-none-eabi/6.3.1/thumb/v7e-m/fpv4-sp/hard/crtn.o
 *(.data*)
 .data._impure_ptr
                0x0000000020000004        0x4 /opt/ti/ccsv7/tools/compiler/gcc-arm-none-eabi-6-2017-q1-update/bin/../lib/gcc/arm-none-eabi/6.3.1/../../../../arm-none-eabi/lib/thumb/v7e-m/fpv4-sp/hard/libc_nano.a(lib_a-impure.o)
                0x0000000020000004                _impure_ptr
 .data.impure_data
                0x0000000020000008       0x60 /opt/ti/ccsv7/tools/compiler/gcc-arm-none-eabi-6-2017-q1-update/bin/../lib/gcc/arm-none-eabi/6.3.1/../../../../arm-none-eabi/lib/thumb/v7e-m/fpv4-sp/hard/libc_nano.a(lib_a-impure.o)
 .data.SystemCoreClock
                0x0000000020000068        0x4 Debug/system_msp432p401r.c.o
                0x0000000020000068                SystemCoreClock
 .data.port_base
                0x000000002000006c       0x28 /home/student/git/workspace_mct/YAHAL/libYAHAL_msp432.a(gpio_msp432.cpp.o)
                0x000000002000006c                port_base
 .data._ZN10__cxxabiv119__terminate_handlerE
                0x0000000020000094        0x4 /opt/ti/ccsv7/tools/compiler/gcc-arm-none-eabi-6-2017-q1-update/bin/../lib/gcc/arm-none-eabi/6.3.1/../../../../arm-none-eabi/lib/thumb/v7e-m/fpv4-sp/hard/libstdc++_nano.a(eh_term_handler.o)
                0x0000000020000094                __cxxabiv1::__terminate_handler
 .data._ZN10__cxxabiv120__unexpected_handlerE
                0x0000000020000098        0x4 /opt/ti/ccsv7/tools/compiler/gcc-arm-none-eabi-6-2017-q1-update/bin/../lib/gcc/arm-none-eabi/6.3.1/../../../../arm-none-eabi/lib/thumb/v7e-m/fpv4-sp/hard/libstdc++_nano.a(eh_unex_handler.o)
                0x0000000020000098                __cxxabiv1::__unexpected_handler
                0x000000002000009c                . = ALIGN (0x4)
                0x000000002000009c                __data_end__ = .

.jcr            0x000000002000009c        0x4 load address 0x0000000000002234
 .jcr           0x000000002000009c        0x0 /opt/ti/ccsv7/tools/compiler/gcc-arm-none-eabi-6-2017-q1-update/bin/../lib/gcc/arm-none-eabi/6.3.1/thumb/v7e-m/fpv4-sp/hard/crtbegin.o
 .jcr           0x000000002000009c        0x4 /opt/ti/ccsv7/tools/compiler/gcc-arm-none-eabi-6-2017-q1-update/bin/../lib/gcc/arm-none-eabi/6.3.1/thumb/v7e-m/fpv4-sp/hard/crtend.o

.igot.plt       0x00000000200000a0        0x0 load address 0x0000000000002238
 .igot.plt      0x00000000200000a0        0x0 /opt/ti/ccsv7/tools/compiler/gcc-arm-none-eabi-6-2017-q1-update/bin/../lib/gcc/arm-none-eabi/6.3.1/thumb/v7e-m/fpv4-sp/hard/crtbegin.o

.bss            0x00000000200000a0      0x240
                0x00000000200000a0                __bss_start__ = .
 *(.shbss)
 *(.bss)
 .bss           0x00000000200000a0        0x0 /opt/ti/ccsv7/tools/compiler/gcc-arm-none-eabi-6-2017-q1-update/bin/../lib/gcc/arm-none-eabi/6.3.1/thumb/v7e-m/fpv4-sp/hard/crti.o
 .bss           0x00000000200000a0       0x1c /opt/ti/ccsv7/tools/compiler/gcc-arm-none-eabi-6-2017-q1-update/bin/../lib/gcc/arm-none-eabi/6.3.1/thumb/v7e-m/fpv4-sp/hard/crtbegin.o
 .bss           0x00000000200000bc        0x0 /opt/ti/ccsv7/tools/compiler/gcc-arm-none-eabi-6-2017-q1-update/bin/../lib/gcc/arm-none-eabi/6.3.1/../../../../arm-none-eabi/lib/thumb/v7e-m/fpv4-sp/hard/crt0.o
 .bss           0x00000000200000bc        0x0 /opt/ti/ccsv7/tools/compiler/gcc-arm-none-eabi-6-2017-q1-update/bin/../lib/gcc/arm-none-eabi/6.3.1/../../../../arm-none-eabi/lib/thumb/v7e-m/fpv4-sp/hard/libc_nano.a(lib_a-exit.o)
 .bss           0x00000000200000bc        0x0 /opt/ti/ccsv7/tools/compiler/gcc-arm-none-eabi-6-2017-q1-update/bin/../lib/gcc/arm-none-eabi/6.3.1/../../../../arm-none-eabi/lib/thumb/v7e-m/fpv4-sp/hard/libc_nano.a(lib_a-impure.o)
 .bss           0x00000000200000bc        0x0 /opt/ti/ccsv7/tools/compiler/gcc-arm-none-eabi-6-2017-q1-update/bin/../lib/gcc/arm-none-eabi/6.3.1/../../../../arm-none-eabi/lib/thumb/v7e-m/fpv4-sp/hard/libc_nano.a(lib_a-init.o)
 .bss           0x00000000200000bc        0x0 /opt/ti/ccsv7/tools/compiler/gcc-arm-none-eabi-6-2017-q1-update/bin/../lib/gcc/arm-none-eabi/6.3.1/../../../../arm-none-eabi/lib/thumb/v7e-m/fpv4-sp/hard/libc_nano.a(lib_a-memset.o)
 .bss           0x00000000200000bc        0x0 /opt/ti/ccsv7/tools/compiler/gcc-arm-none-eabi-6-2017-q1-update/bin/../lib/gcc/arm-none-eabi/6.3.1/../../../../arm-none-eabi/lib/thumb/v7e-m/fpv4-sp/hard/libnosys.a(_exit.o)
 .bss           0x00000000200000bc        0x0 Debug/main.cpp.o
 .bss           0x00000000200000bc        0x0 Debug/startup_msp432p401r_gcc.c.o
 .bss           0x00000000200000bc        0x0 Debug/system_msp432p401r.c.o
 .bss           0x00000000200000bc        0x0 /home/student/git/workspace_mct/YAHAL/libYAHAL_msp432.a(gpio_msp432.cpp.o)
 .bss           0x00000000200000bc        0x0 /home/student/git/workspace_mct/YAHAL/libYAHAL_msp432.a(timer_msp432.cpp.o)
 .bss           0x00000000200000bc        0x0 /opt/ti/ccsv7/tools/compiler/gcc-arm-none-eabi-6-2017-q1-update/bin/../lib/gcc/arm-none-eabi/6.3.1/../../../../arm-none-eabi/lib/thumb/v7e-m/fpv4-sp/hard/libstdc++_nano.a(class_type_info.o)
 .bss           0x00000000200000bc        0x0 /opt/ti/ccsv7/tools/compiler/gcc-arm-none-eabi-6-2017-q1-update/bin/../lib/gcc/arm-none-eabi/6.3.1/../../../../arm-none-eabi/lib/thumb/v7e-m/fpv4-sp/hard/libstdc++_nano.a(atexit_arm.o)
 .bss           0x00000000200000bc        0x0 /opt/ti/ccsv7/tools/compiler/gcc-arm-none-eabi-6-2017-q1-update/bin/../lib/gcc/arm-none-eabi/6.3.1/../../../../arm-none-eabi/lib/thumb/v7e-m/fpv4-sp/hard/libstdc++_nano.a(si_class_type_info.o)
 .bss           0x00000000200000bc        0x0 /opt/ti/ccsv7/tools/compiler/gcc-arm-none-eabi-6-2017-q1-update/bin/../lib/gcc/arm-none-eabi/6.3.1/../../../../arm-none-eabi/lib/thumb/v7e-m/fpv4-sp/hard/libstdc++_nano.a(del_ops.o)
 .bss           0x00000000200000bc        0x0 /opt/ti/ccsv7/tools/compiler/gcc-arm-none-eabi-6-2017-q1-update/bin/../lib/gcc/arm-none-eabi/6.3.1/../../../../arm-none-eabi/lib/thumb/v7e-m/fpv4-sp/hard/libstdc++_nano.a(del_op.o)
 .bss           0x00000000200000bc        0x0 /opt/ti/ccsv7/tools/compiler/gcc-arm-none-eabi-6-2017-q1-update/bin/../lib/gcc/arm-none-eabi/6.3.1/../../../../arm-none-eabi/lib/thumb/v7e-m/fpv4-sp/hard/libstdc++_nano.a(pure.o)
 .bss           0x00000000200000bc        0x0 /opt/ti/ccsv7/tools/compiler/gcc-arm-none-eabi-6-2017-q1-update/bin/../lib/gcc/arm-none-eabi/6.3.1/../../../../arm-none-eabi/lib/thumb/v7e-m/fpv4-sp/hard/libstdc++_nano.a(tinfo.o)
 .bss           0x00000000200000bc        0x0 /opt/ti/ccsv7/tools/compiler/gcc-arm-none-eabi-6-2017-q1-update/bin/../lib/gcc/arm-none-eabi/6.3.1/../../../../arm-none-eabi/lib/thumb/v7e-m/fpv4-sp/hard/libstdc++_nano.a(eh_terminate.o)
 .bss           0x00000000200000bc        0x0 /opt/ti/ccsv7/tools/compiler/gcc-arm-none-eabi-6-2017-q1-update/bin/../lib/gcc/arm-none-eabi/6.3.1/../../../../arm-none-eabi/lib/thumb/v7e-m/fpv4-sp/hard/libstdc++_nano.a(eh_term_handler.o)
 .bss           0x00000000200000bc        0x0 /opt/ti/ccsv7/tools/compiler/gcc-arm-none-eabi-6-2017-q1-update/bin/../lib/gcc/arm-none-eabi/6.3.1/../../../../arm-none-eabi/lib/thumb/v7e-m/fpv4-sp/hard/libstdc++_nano.a(eh_unex_handler.o)
 .bss           0x00000000200000bc        0x0 /opt/ti/ccsv7/tools/compiler/gcc-arm-none-eabi-6-2017-q1-update/bin/../lib/gcc/arm-none-eabi/6.3.1/../../../../arm-none-eabi/lib/thumb/v7e-m/fpv4-sp/hard/libc_nano.a(lib_a-abort.o)
 .bss           0x00000000200000bc        0x0 /opt/ti/ccsv7/tools/compiler/gcc-arm-none-eabi-6-2017-q1-update/bin/../lib/gcc/arm-none-eabi/6.3.1/../../../../arm-none-eabi/lib/thumb/v7e-m/fpv4-sp/hard/libc_nano.a(lib_a-cxa_atexit.o)
 .bss           0x00000000200000bc        0x0 /opt/ti/ccsv7/tools/compiler/gcc-arm-none-eabi-6-2017-q1-update/bin/../lib/gcc/arm-none-eabi/6.3.1/../../../../arm-none-eabi/lib/thumb/v7e-m/fpv4-sp/hard/libc_nano.a(lib_a-malloc.o)
 .bss           0x00000000200000bc        0x0 /opt/ti/ccsv7/tools/compiler/gcc-arm-none-eabi-6-2017-q1-update/bin/../lib/gcc/arm-none-eabi/6.3.1/../../../../arm-none-eabi/lib/thumb/v7e-m/fpv4-sp/hard/libc_nano.a(lib_a-nano-freer.o)
 .bss           0x00000000200000bc        0x0 /opt/ti/ccsv7/tools/compiler/gcc-arm-none-eabi-6-2017-q1-update/bin/../lib/gcc/arm-none-eabi/6.3.1/../../../../arm-none-eabi/lib/thumb/v7e-m/fpv4-sp/hard/libc_nano.a(lib_a-nano-mallocr.o)
 .bss           0x00000000200000bc        0x0 /opt/ti/ccsv7/tools/compiler/gcc-arm-none-eabi-6-2017-q1-update/bin/../lib/gcc/arm-none-eabi/6.3.1/../../../../arm-none-eabi/lib/thumb/v7e-m/fpv4-sp/hard/libc_nano.a(lib_a-on_exit_args.o)
 .bss           0x00000000200000bc        0x0 /opt/ti/ccsv7/tools/compiler/gcc-arm-none-eabi-6-2017-q1-update/bin/../lib/gcc/arm-none-eabi/6.3.1/../../../../arm-none-eabi/lib/thumb/v7e-m/fpv4-sp/hard/libc_nano.a(lib_a-sbrkr.o)
 .bss           0x00000000200000bc        0x0 /opt/ti/ccsv7/tools/compiler/gcc-arm-none-eabi-6-2017-q1-update/bin/../lib/gcc/arm-none-eabi/6.3.1/../../../../arm-none-eabi/lib/thumb/v7e-m/fpv4-sp/hard/libc_nano.a(lib_a-signal.o)
 .bss           0x00000000200000bc        0x0 /opt/ti/ccsv7/tools/compiler/gcc-arm-none-eabi-6-2017-q1-update/bin/../lib/gcc/arm-none-eabi/6.3.1/../../../../arm-none-eabi/lib/thumb/v7e-m/fpv4-sp/hard/libc_nano.a(lib_a-signalr.o)
 .bss           0x00000000200000bc        0x0 /opt/ti/ccsv7/tools/compiler/gcc-arm-none-eabi-6-2017-q1-update/bin/../lib/gcc/arm-none-eabi/6.3.1/../../../../arm-none-eabi/lib/thumb/v7e-m/fpv4-sp/hard/libc_nano.a(lib_a-strcmp.o)
 .bss           0x00000000200000bc        0x0 /opt/ti/ccsv7/tools/compiler/gcc-arm-none-eabi-6-2017-q1-update/bin/../lib/gcc/arm-none-eabi/6.3.1/../../../../arm-none-eabi/lib/thumb/v7e-m/fpv4-sp/hard/libc_nano.a(lib_a-mlock.o)
 .bss           0x00000000200000bc        0x0 /opt/ti/ccsv7/tools/compiler/gcc-arm-none-eabi-6-2017-q1-update/bin/../lib/gcc/arm-none-eabi/6.3.1/../../../../arm-none-eabi/lib/thumb/v7e-m/fpv4-sp/hard/libc_nano.a(lib_a-reent.o)
 .bss           0x00000000200000bc        0x0 /opt/ti/ccsv7/tools/compiler/gcc-arm-none-eabi-6-2017-q1-update/bin/../lib/gcc/arm-none-eabi/6.3.1/../../../../arm-none-eabi/lib/thumb/v7e-m/fpv4-sp/hard/libnosys.a(getpid.o)
 .bss           0x00000000200000bc        0x0 /opt/ti/ccsv7/tools/compiler/gcc-arm-none-eabi-6-2017-q1-update/bin/../lib/gcc/arm-none-eabi/6.3.1/../../../../arm-none-eabi/lib/thumb/v7e-m/fpv4-sp/hard/libnosys.a(kill.o)
 .bss           0x00000000200000bc        0x0 /opt/ti/ccsv7/tools/compiler/gcc-arm-none-eabi-6-2017-q1-update/bin/../lib/gcc/arm-none-eabi/6.3.1/../../../../arm-none-eabi/lib/thumb/v7e-m/fpv4-sp/hard/libnosys.a(sbrk.o)
 .bss           0x00000000200000bc        0x0 /opt/ti/ccsv7/tools/compiler/gcc-arm-none-eabi-6-2017-q1-update/bin/../lib/gcc/arm-none-eabi/6.3.1/thumb/v7e-m/fpv4-sp/hard/crtend.o
 .bss           0x00000000200000bc        0x0 /opt/ti/ccsv7/tools/compiler/gcc-arm-none-eabi-6-2017-q1-update/bin/../lib/gcc/arm-none-eabi/6.3.1/thumb/v7e-m/fpv4-sp/hard/crtn.o
 *(.bss.*)
 .bss._ZL17yahal_assert_file
                0x00000000200000bc        0x4 /home/student/git/workspace_mct/YAHAL/libYAHAL_msp432.a(gpio_msp432.cpp.o)
 .bss._ZL17yahal_assert_line
                0x00000000200000c0        0x4 /home/student/git/workspace_mct/YAHAL/libYAHAL_msp432.a(gpio_msp432.cpp.o)
 .bss._ZN11gpio_msp4324instE
                0x00000000200000c4       0xec /home/student/git/workspace_mct/YAHAL/libYAHAL_msp432.a(gpio_msp432.cpp.o)
                0x00000000200000c4                gpio_msp432::inst
 .bss._ZL17yahal_assert_file
                0x00000000200001b0        0x4 /home/student/git/workspace_mct/YAHAL/libYAHAL_msp432.a(timer_msp432.cpp.o)
 .bss._ZL17yahal_assert_line
                0x00000000200001b4        0x4 /home/student/git/workspace_mct/YAHAL/libYAHAL_msp432.a(timer_msp432.cpp.o)
 .bss._ZN12timer_msp43212_intHandler1E
                0x00000000200001b8        0x4 /home/student/git/workspace_mct/YAHAL/libYAHAL_msp432.a(timer_msp432.cpp.o)
                0x00000000200001b8                timer_msp432::_intHandler1
 .bss._ZN12timer_msp43212_intHandler2E
                0x00000000200001bc        0x4 /home/student/git/workspace_mct/YAHAL/libYAHAL_msp432.a(timer_msp432.cpp.o)
                0x00000000200001bc                timer_msp432::_intHandler2
 .bss._ZN12timer_msp4325_arg1E
                0x00000000200001c0        0x4 /home/student/git/workspace_mct/YAHAL/libYAHAL_msp432.a(timer_msp432.cpp.o)
                0x00000000200001c0                timer_msp432::_arg1
 .bss._ZN12timer_msp4325_arg2E
                0x00000000200001c4        0x4 /home/student/git/workspace_mct/YAHAL/libYAHAL_msp432.a(timer_msp432.cpp.o)
                0x00000000200001c4                timer_msp432::_arg2
 .bss.__malloc_free_list
                0x00000000200001c8        0x4 /opt/ti/ccsv7/tools/compiler/gcc-arm-none-eabi-6-2017-q1-update/bin/../lib/gcc/arm-none-eabi/6.3.1/../../../../arm-none-eabi/lib/thumb/v7e-m/fpv4-sp/hard/libc_nano.a(lib_a-nano-mallocr.o)
                0x00000000200001c8                __malloc_free_list
 .bss.__malloc_sbrk_start
                0x00000000200001cc        0x4 /opt/ti/ccsv7/tools/compiler/gcc-arm-none-eabi-6-2017-q1-update/bin/../lib/gcc/arm-none-eabi/6.3.1/../../../../arm-none-eabi/lib/thumb/v7e-m/fpv4-sp/hard/libc_nano.a(lib_a-nano-mallocr.o)
                0x00000000200001cc                __malloc_sbrk_start
 .bss._on_exit_args_instance
                0x00000000200001d0      0x108 /opt/ti/ccsv7/tools/compiler/gcc-arm-none-eabi-6-2017-q1-update/bin/../lib/gcc/arm-none-eabi/6.3.1/../../../../arm-none-eabi/lib/thumb/v7e-m/fpv4-sp/hard/libc_nano.a(lib_a-on_exit_args.o)
 .bss.heap_end.5239
                0x00000000200002d8        0x4 /opt/ti/ccsv7/tools/compiler/gcc-arm-none-eabi-6-2017-q1-update/bin/../lib/gcc/arm-none-eabi/6.3.1/../../../../arm-none-eabi/lib/thumb/v7e-m/fpv4-sp/hard/libnosys.a(sbrk.o)
 *(COMMON)
 COMMON         0x00000000200002dc        0x4 /opt/ti/ccsv7/tools/compiler/gcc-arm-none-eabi-6-2017-q1-update/bin/../lib/gcc/arm-none-eabi/6.3.1/../../../../arm-none-eabi/lib/thumb/v7e-m/fpv4-sp/hard/libc_nano.a(lib_a-reent.o)
                0x00000000200002dc                errno
                0x00000000200002e0                . = ALIGN (0x4)
                0x00000000200002e0                __bss_end__ = .

.heap           0x00000000200002e0        0x0
                0x00000000200002e0                __heap_start__ = .
                0x00000000200002e0                end = __heap_start__
                0x00000000200002e0                _end = end
                0x00000000200002e0                __end = end
 *(.heap)
                0x00000000200002e0                __heap_end__ = .
                0x00000000200002e0                __HeapLimit = __heap_end__

.stack          0x00000000200002e0        0x0
                0x00000000200002e0                _stack = .
 *(.stack)
                0x0000000020010000                __StackTop = (ORIGIN (REGION_STACK) + LENGTH (REGION_STACK))
                0x0000000020010000                PROVIDE (__stack, __StackTop)
LOAD /opt/ti/ccsv7/tools/compiler/gcc-arm-none-eabi-6-2017-q1-update/bin/../lib/gcc/arm-none-eabi/6.3.1/../../../../arm-none-eabi/lib/thumb/v7e-m/fpv4-sp/hard/libstdc++_nano.a
LOAD /opt/ti/ccsv7/tools/compiler/gcc-arm-none-eabi-6-2017-q1-update/bin/../lib/gcc/arm-none-eabi/6.3.1/thumb/v7e-m/fpv4-sp/hard/libgcc.a
LOAD /opt/ti/ccsv7/tools/compiler/gcc-arm-none-eabi-6-2017-q1-update/bin/../lib/gcc/arm-none-eabi/6.3.1/../../../../arm-none-eabi/lib/thumb/v7e-m/fpv4-sp/hard/libc_nano.a
LOAD /opt/ti/ccsv7/tools/compiler/gcc-arm-none-eabi-6-2017-q1-update/bin/../lib/gcc/arm-none-eabi/6.3.1/../../../../arm-none-eabi/lib/thumb/v7e-m/fpv4-sp/hard/libnosys.a
START GROUP
LOAD Debug/main.cpp.o
LOAD Debug/startup_msp432p401r_gcc.c.o
LOAD Debug/system_msp432p401r.c.o
LOAD /home/student/git/workspace_mct/YAHAL/libYAHAL_msp432.a
LOAD /opt/ti/ccsv7/tools/compiler/gcc-arm-none-eabi-6-2017-q1-update/bin/../lib/gcc/arm-none-eabi/6.3.1/../../../../arm-none-eabi/lib/thumb/v7e-m/fpv4-sp/hard/libstdc++_nano.a
LOAD /opt/ti/ccsv7/tools/compiler/gcc-arm-none-eabi-6-2017-q1-update/bin/../lib/gcc/arm-none-eabi/6.3.1/thumb/v7e-m/fpv4-sp/hard/libgcc.a
LOAD /opt/ti/ccsv7/tools/compiler/gcc-arm-none-eabi-6-2017-q1-update/bin/../lib/gcc/arm-none-eabi/6.3.1/../../../../arm-none-eabi/lib/thumb/v7e-m/fpv4-sp/hard/libc_nano.a
LOAD /opt/ti/ccsv7/tools/compiler/gcc-arm-none-eabi-6-2017-q1-update/bin/../lib/gcc/arm-none-eabi/6.3.1/../../../../arm-none-eabi/lib/thumb/v7e-m/fpv4-sp/hard/libm.a
LOAD /opt/ti/ccsv7/tools/compiler/gcc-arm-none-eabi-6-2017-q1-update/bin/../lib/gcc/arm-none-eabi/6.3.1/../../../../arm-none-eabi/lib/thumb/v7e-m/fpv4-sp/hard/libnosys.a
END GROUP
LOAD /opt/ti/ccsv7/tools/compiler/gcc-arm-none-eabi-6-2017-q1-update/bin/../lib/gcc/arm-none-eabi/6.3.1/../../../../arm-none-eabi/lib/thumb/v7e-m/fpv4-sp/hard/libstdc++.a
LOAD /opt/ti/ccsv7/tools/compiler/gcc-arm-none-eabi-6-2017-q1-update/bin/../lib/gcc/arm-none-eabi/6.3.1/../../../../arm-none-eabi/lib/thumb/v7e-m/fpv4-sp/hard/libm.a
START GROUP
LOAD /opt/ti/ccsv7/tools/compiler/gcc-arm-none-eabi-6-2017-q1-update/bin/../lib/gcc/arm-none-eabi/6.3.1/thumb/v7e-m/fpv4-sp/hard/libgcc.a
LOAD /opt/ti/ccsv7/tools/compiler/gcc-arm-none-eabi-6-2017-q1-update/bin/../lib/gcc/arm-none-eabi/6.3.1/../../../../arm-none-eabi/lib/thumb/v7e-m/fpv4-sp/hard/libg.a
LOAD /opt/ti/ccsv7/tools/compiler/gcc-arm-none-eabi-6-2017-q1-update/bin/../lib/gcc/arm-none-eabi/6.3.1/../../../../arm-none-eabi/lib/thumb/v7e-m/fpv4-sp/hard/libc.a
END GROUP
LOAD /opt/ti/ccsv7/tools/compiler/gcc-arm-none-eabi-6-2017-q1-update/bin/../lib/gcc/arm-none-eabi/6.3.1/thumb/v7e-m/fpv4-sp/hard/crtend.o
LOAD /opt/ti/ccsv7/tools/compiler/gcc-arm-none-eabi-6-2017-q1-update/bin/../lib/gcc/arm-none-eabi/6.3.1/thumb/v7e-m/fpv4-sp/hard/crtn.o
OUTPUT(example_blink_timer.out elf32-littlearm)

.ARM.attributes
                0x0000000000000000       0x30
 .ARM.attributes
                0x0000000000000000       0x22 /opt/ti/ccsv7/tools/compiler/gcc-arm-none-eabi-6-2017-q1-update/bin/../lib/gcc/arm-none-eabi/6.3.1/thumb/v7e-m/fpv4-sp/hard/crti.o
 .ARM.attributes
                0x0000000000000022       0x34 /opt/ti/ccsv7/tools/compiler/gcc-arm-none-eabi-6-2017-q1-update/bin/../lib/gcc/arm-none-eabi/6.3.1/thumb/v7e-m/fpv4-sp/hard/crtbegin.o
 .ARM.attributes
                0x0000000000000056       0x20 /opt/ti/ccsv7/tools/compiler/gcc-arm-none-eabi-6-2017-q1-update/bin/../lib/gcc/arm-none-eabi/6.3.1/../../../../arm-none-eabi/lib/thumb/v7e-m/fpv4-sp/hard/crt0.o
 .ARM.attributes
                0x0000000000000076       0x34 /opt/ti/ccsv7/tools/compiler/gcc-arm-none-eabi-6-2017-q1-update/bin/../lib/gcc/arm-none-eabi/6.3.1/../../../../arm-none-eabi/lib/thumb/v7e-m/fpv4-sp/hard/libc_nano.a(lib_a-exit.o)
 .ARM.attributes
                0x00000000000000aa       0x34 /opt/ti/ccsv7/tools/compiler/gcc-arm-none-eabi-6-2017-q1-update/bin/../lib/gcc/arm-none-eabi/6.3.1/../../../../arm-none-eabi/lib/thumb/v7e-m/fpv4-sp/hard/libc_nano.a(lib_a-impure.o)
 .ARM.attributes
                0x00000000000000de       0x34 /opt/ti/ccsv7/tools/compiler/gcc-arm-none-eabi-6-2017-q1-update/bin/../lib/gcc/arm-none-eabi/6.3.1/../../../../arm-none-eabi/lib/thumb/v7e-m/fpv4-sp/hard/libc_nano.a(lib_a-init.o)
 .ARM.attributes
                0x0000000000000112       0x34 /opt/ti/ccsv7/tools/compiler/gcc-arm-none-eabi-6-2017-q1-update/bin/../lib/gcc/arm-none-eabi/6.3.1/../../../../arm-none-eabi/lib/thumb/v7e-m/fpv4-sp/hard/libc_nano.a(lib_a-memset.o)
 .ARM.attributes
                0x0000000000000146       0x34 /opt/ti/ccsv7/tools/compiler/gcc-arm-none-eabi-6-2017-q1-update/bin/../lib/gcc/arm-none-eabi/6.3.1/../../../../arm-none-eabi/lib/thumb/v7e-m/fpv4-sp/hard/libnosys.a(_exit.o)
 .ARM.attributes
                0x000000000000017a       0x39 Debug/main.cpp.o
 .ARM.attributes
                0x00000000000001b3       0x39 Debug/startup_msp432p401r_gcc.c.o
 .ARM.attributes
                0x00000000000001ec       0x39 Debug/system_msp432p401r.c.o
 .ARM.attributes
                0x0000000000000225       0x39 /home/student/git/workspace_mct/YAHAL/libYAHAL_msp432.a(gpio_msp432.cpp.o)
 .ARM.attributes
                0x000000000000025e       0x39 /home/student/git/workspace_mct/YAHAL/libYAHAL_msp432.a(timer_msp432.cpp.o)
 .ARM.attributes
                0x0000000000000297       0x34 /opt/ti/ccsv7/tools/compiler/gcc-arm-none-eabi-6-2017-q1-update/bin/../lib/gcc/arm-none-eabi/6.3.1/../../../../arm-none-eabi/lib/thumb/v7e-m/fpv4-sp/hard/libstdc++_nano.a(class_type_info.o)
 .ARM.attributes
                0x00000000000002cb       0x34 /opt/ti/ccsv7/tools/compiler/gcc-arm-none-eabi-6-2017-q1-update/bin/../lib/gcc/arm-none-eabi/6.3.1/../../../../arm-none-eabi/lib/thumb/v7e-m/fpv4-sp/hard/libstdc++_nano.a(atexit_arm.o)
 .ARM.attributes
                0x00000000000002ff       0x34 /opt/ti/ccsv7/tools/compiler/gcc-arm-none-eabi-6-2017-q1-update/bin/../lib/gcc/arm-none-eabi/6.3.1/../../../../arm-none-eabi/lib/thumb/v7e-m/fpv4-sp/hard/libstdc++_nano.a(si_class_type_info.o)
 .ARM.attributes
                0x0000000000000333       0x34 /opt/ti/ccsv7/tools/compiler/gcc-arm-none-eabi-6-2017-q1-update/bin/../lib/gcc/arm-none-eabi/6.3.1/../../../../arm-none-eabi/lib/thumb/v7e-m/fpv4-sp/hard/libstdc++_nano.a(del_ops.o)
 .ARM.attributes
                0x0000000000000367       0x34 /opt/ti/ccsv7/tools/compiler/gcc-arm-none-eabi-6-2017-q1-update/bin/../lib/gcc/arm-none-eabi/6.3.1/../../../../arm-none-eabi/lib/thumb/v7e-m/fpv4-sp/hard/libstdc++_nano.a(del_op.o)
 .ARM.attributes
                0x000000000000039b       0x34 /opt/ti/ccsv7/tools/compiler/gcc-arm-none-eabi-6-2017-q1-update/bin/../lib/gcc/arm-none-eabi/6.3.1/../../../../arm-none-eabi/lib/thumb/v7e-m/fpv4-sp/hard/libstdc++_nano.a(pure.o)
 .ARM.attributes
                0x00000000000003cf       0x34 /opt/ti/ccsv7/tools/compiler/gcc-arm-none-eabi-6-2017-q1-update/bin/../lib/gcc/arm-none-eabi/6.3.1/../../../../arm-none-eabi/lib/thumb/v7e-m/fpv4-sp/hard/libstdc++_nano.a(tinfo.o)
 .ARM.attributes
                0x0000000000000403       0x34 /opt/ti/ccsv7/tools/compiler/gcc-arm-none-eabi-6-2017-q1-update/bin/../lib/gcc/arm-none-eabi/6.3.1/../../../../arm-none-eabi/lib/thumb/v7e-m/fpv4-sp/hard/libstdc++_nano.a(eh_terminate.o)
 .ARM.attributes
                0x0000000000000437       0x34 /opt/ti/ccsv7/tools/compiler/gcc-arm-none-eabi-6-2017-q1-update/bin/../lib/gcc/arm-none-eabi/6.3.1/../../../../arm-none-eabi/lib/thumb/v7e-m/fpv4-sp/hard/libstdc++_nano.a(eh_term_handler.o)
 .ARM.attributes
                0x000000000000046b       0x34 /opt/ti/ccsv7/tools/compiler/gcc-arm-none-eabi-6-2017-q1-update/bin/../lib/gcc/arm-none-eabi/6.3.1/../../../../arm-none-eabi/lib/thumb/v7e-m/fpv4-sp/hard/libstdc++_nano.a(eh_unex_handler.o)
 .ARM.attributes
                0x000000000000049f       0x34 /opt/ti/ccsv7/tools/compiler/gcc-arm-none-eabi-6-2017-q1-update/bin/../lib/gcc/arm-none-eabi/6.3.1/../../../../arm-none-eabi/lib/thumb/v7e-m/fpv4-sp/hard/libc_nano.a(lib_a-abort.o)
 .ARM.attributes
                0x00000000000004d3       0x34 /opt/ti/ccsv7/tools/compiler/gcc-arm-none-eabi-6-2017-q1-update/bin/../lib/gcc/arm-none-eabi/6.3.1/../../../../arm-none-eabi/lib/thumb/v7e-m/fpv4-sp/hard/libc_nano.a(lib_a-cxa_atexit.o)
 .ARM.attributes
                0x0000000000000507       0x34 /opt/ti/ccsv7/tools/compiler/gcc-arm-none-eabi-6-2017-q1-update/bin/../lib/gcc/arm-none-eabi/6.3.1/../../../../arm-none-eabi/lib/thumb/v7e-m/fpv4-sp/hard/libc_nano.a(lib_a-malloc.o)
 .ARM.attributes
                0x000000000000053b       0x34 /opt/ti/ccsv7/tools/compiler/gcc-arm-none-eabi-6-2017-q1-update/bin/../lib/gcc/arm-none-eabi/6.3.1/../../../../arm-none-eabi/lib/thumb/v7e-m/fpv4-sp/hard/libc_nano.a(lib_a-nano-freer.o)
 .ARM.attributes
                0x000000000000056f       0x34 /opt/ti/ccsv7/tools/compiler/gcc-arm-none-eabi-6-2017-q1-update/bin/../lib/gcc/arm-none-eabi/6.3.1/../../../../arm-none-eabi/lib/thumb/v7e-m/fpv4-sp/hard/libc_nano.a(lib_a-nano-mallocr.o)
 .ARM.attributes
                0x00000000000005a3       0x34 /opt/ti/ccsv7/tools/compiler/gcc-arm-none-eabi-6-2017-q1-update/bin/../lib/gcc/arm-none-eabi/6.3.1/../../../../arm-none-eabi/lib/thumb/v7e-m/fpv4-sp/hard/libc_nano.a(lib_a-on_exit_args.o)
 .ARM.attributes
                0x00000000000005d7       0x34 /opt/ti/ccsv7/tools/compiler/gcc-arm-none-eabi-6-2017-q1-update/bin/../lib/gcc/arm-none-eabi/6.3.1/../../../../arm-none-eabi/lib/thumb/v7e-m/fpv4-sp/hard/libc_nano.a(lib_a-sbrkr.o)
 .ARM.attributes
                0x000000000000060b       0x34 /opt/ti/ccsv7/tools/compiler/gcc-arm-none-eabi-6-2017-q1-update/bin/../lib/gcc/arm-none-eabi/6.3.1/../../../../arm-none-eabi/lib/thumb/v7e-m/fpv4-sp/hard/libc_nano.a(lib_a-signal.o)
 .ARM.attributes
                0x000000000000063f       0x34 /opt/ti/ccsv7/tools/compiler/gcc-arm-none-eabi-6-2017-q1-update/bin/../lib/gcc/arm-none-eabi/6.3.1/../../../../arm-none-eabi/lib/thumb/v7e-m/fpv4-sp/hard/libc_nano.a(lib_a-signalr.o)
 .ARM.attributes
                0x0000000000000673       0x20 /opt/ti/ccsv7/tools/compiler/gcc-arm-none-eabi-6-2017-q1-update/bin/../lib/gcc/arm-none-eabi/6.3.1/../../../../arm-none-eabi/lib/thumb/v7e-m/fpv4-sp/hard/libc_nano.a(lib_a-strcmp.o)
 .ARM.attributes
                0x0000000000000693       0x34 /opt/ti/ccsv7/tools/compiler/gcc-arm-none-eabi-6-2017-q1-update/bin/../lib/gcc/arm-none-eabi/6.3.1/../../../../arm-none-eabi/lib/thumb/v7e-m/fpv4-sp/hard/libc_nano.a(lib_a-mlock.o)
 .ARM.attributes
                0x00000000000006c7       0x34 /opt/ti/ccsv7/tools/compiler/gcc-arm-none-eabi-6-2017-q1-update/bin/../lib/gcc/arm-none-eabi/6.3.1/../../../../arm-none-eabi/lib/thumb/v7e-m/fpv4-sp/hard/libc_nano.a(lib_a-reent.o)
 .ARM.attributes
                0x00000000000006fb       0x34 /opt/ti/ccsv7/tools/compiler/gcc-arm-none-eabi-6-2017-q1-update/bin/../lib/gcc/arm-none-eabi/6.3.1/../../../../arm-none-eabi/lib/thumb/v7e-m/fpv4-sp/hard/libnosys.a(getpid.o)
 .ARM.attributes
                0x000000000000072f       0x34 /opt/ti/ccsv7/tools/compiler/gcc-arm-none-eabi-6-2017-q1-update/bin/../lib/gcc/arm-none-eabi/6.3.1/../../../../arm-none-eabi/lib/thumb/v7e-m/fpv4-sp/hard/libnosys.a(kill.o)
 .ARM.attributes
                0x0000000000000763       0x34 /opt/ti/ccsv7/tools/compiler/gcc-arm-none-eabi-6-2017-q1-update/bin/../lib/gcc/arm-none-eabi/6.3.1/../../../../arm-none-eabi/lib/thumb/v7e-m/fpv4-sp/hard/libnosys.a(sbrk.o)
 .ARM.attributes
                0x0000000000000797       0x34 /opt/ti/ccsv7/tools/compiler/gcc-arm-none-eabi-6-2017-q1-update/bin/../lib/gcc/arm-none-eabi/6.3.1/thumb/v7e-m/fpv4-sp/hard/crtend.o
 .ARM.attributes
                0x00000000000007cb       0x22 /opt/ti/ccsv7/tools/compiler/gcc-arm-none-eabi-6-2017-q1-update/bin/../lib/gcc/arm-none-eabi/6.3.1/thumb/v7e-m/fpv4-sp/hard/crtn.o

.comment        0x0000000000000000       0x7f
 .comment       0x0000000000000000       0x7f Debug/main.cpp.o
                                         0x80 (size before relaxing)
 .comment       0x000000000000007f       0x80 Debug/startup_msp432p401r_gcc.c.o
 .comment       0x000000000000007f       0x80 Debug/system_msp432p401r.c.o
 .comment       0x000000000000007f       0x80 /home/student/git/workspace_mct/YAHAL/libYAHAL_msp432.a(gpio_msp432.cpp.o)
 .comment       0x000000000000007f       0x80 /home/student/git/workspace_mct/YAHAL/libYAHAL_msp432.a(timer_msp432.cpp.o)

.debug_frame    0x0000000000000000      0xfbc
 .debug_frame   0x0000000000000000       0x28 /opt/ti/ccsv7/tools/compiler/gcc-arm-none-eabi-6-2017-q1-update/bin/../lib/gcc/arm-none-eabi/6.3.1/../../../../arm-none-eabi/lib/thumb/v7e-m/fpv4-sp/hard/libc_nano.a(lib_a-exit.o)
 .debug_frame   0x0000000000000028       0x2c /opt/ti/ccsv7/tools/compiler/gcc-arm-none-eabi-6-2017-q1-update/bin/../lib/gcc/arm-none-eabi/6.3.1/../../../../arm-none-eabi/lib/thumb/v7e-m/fpv4-sp/hard/libc_nano.a(lib_a-init.o)
 .debug_frame   0x0000000000000054       0x20 /opt/ti/ccsv7/tools/compiler/gcc-arm-none-eabi-6-2017-q1-update/bin/../lib/gcc/arm-none-eabi/6.3.1/../../../../arm-none-eabi/lib/thumb/v7e-m/fpv4-sp/hard/libc_nano.a(lib_a-memset.o)
 .debug_frame   0x0000000000000074       0x20 /opt/ti/ccsv7/tools/compiler/gcc-arm-none-eabi-6-2017-q1-update/bin/../lib/gcc/arm-none-eabi/6.3.1/../../../../arm-none-eabi/lib/thumb/v7e-m/fpv4-sp/hard/libnosys.a(_exit.o)
 .debug_frame   0x0000000000000094      0x158 Debug/main.cpp.o
 .debug_frame   0x00000000000001ec       0x4c Debug/startup_msp432p401r_gcc.c.o
 .debug_frame   0x0000000000000238       0x58 Debug/system_msp432p401r.c.o
 .debug_frame   0x0000000000000290      0x3dc /home/student/git/workspace_mct/YAHAL/libYAHAL_msp432.a(gpio_msp432.cpp.o)
 .debug_frame   0x000000000000066c      0x2ac /home/student/git/workspace_mct/YAHAL/libYAHAL_msp432.a(timer_msp432.cpp.o)
 .debug_frame   0x0000000000000918       0xd8 /opt/ti/ccsv7/tools/compiler/gcc-arm-none-eabi-6-2017-q1-update/bin/../lib/gcc/arm-none-eabi/6.3.1/../../../../arm-none-eabi/lib/thumb/v7e-m/fpv4-sp/hard/libstdc++_nano.a(class_type_info.o)
 .debug_frame   0x00000000000009f0       0x20 /opt/ti/ccsv7/tools/compiler/gcc-arm-none-eabi-6-2017-q1-update/bin/../lib/gcc/arm-none-eabi/6.3.1/../../../../arm-none-eabi/lib/thumb/v7e-m/fpv4-sp/hard/libstdc++_nano.a(atexit_arm.o)
 .debug_frame   0x0000000000000a10       0xd8 /opt/ti/ccsv7/tools/compiler/gcc-arm-none-eabi-6-2017-q1-update/bin/../lib/gcc/arm-none-eabi/6.3.1/../../../../arm-none-eabi/lib/thumb/v7e-m/fpv4-sp/hard/libstdc++_nano.a(si_class_type_info.o)
 .debug_frame   0x0000000000000ae8       0x20 /opt/ti/ccsv7/tools/compiler/gcc-arm-none-eabi-6-2017-q1-update/bin/../lib/gcc/arm-none-eabi/6.3.1/../../../../arm-none-eabi/lib/thumb/v7e-m/fpv4-sp/hard/libstdc++_nano.a(del_ops.o)
 .debug_frame   0x0000000000000b08       0x20 /opt/ti/ccsv7/tools/compiler/gcc-arm-none-eabi-6-2017-q1-update/bin/../lib/gcc/arm-none-eabi/6.3.1/../../../../arm-none-eabi/lib/thumb/v7e-m/fpv4-sp/hard/libstdc++_nano.a(del_op.o)
 .debug_frame   0x0000000000000b28       0x40 /opt/ti/ccsv7/tools/compiler/gcc-arm-none-eabi-6-2017-q1-update/bin/../lib/gcc/arm-none-eabi/6.3.1/../../../../arm-none-eabi/lib/thumb/v7e-m/fpv4-sp/hard/libstdc++_nano.a(pure.o)
 .debug_frame   0x0000000000000b68       0x80 /opt/ti/ccsv7/tools/compiler/gcc-arm-none-eabi-6-2017-q1-update/bin/../lib/gcc/arm-none-eabi/6.3.1/../../../../arm-none-eabi/lib/thumb/v7e-m/fpv4-sp/hard/libstdc++_nano.a(tinfo.o)
 .debug_frame   0x0000000000000be8       0xb0 /opt/ti/ccsv7/tools/compiler/gcc-arm-none-eabi-6-2017-q1-update/bin/../lib/gcc/arm-none-eabi/6.3.1/../../../../arm-none-eabi/lib/thumb/v7e-m/fpv4-sp/hard/libstdc++_nano.a(eh_terminate.o)
 .debug_frame   0x0000000000000c98       0x28 /opt/ti/ccsv7/tools/compiler/gcc-arm-none-eabi-6-2017-q1-update/bin/../lib/gcc/arm-none-eabi/6.3.1/../../../../arm-none-eabi/lib/thumb/v7e-m/fpv4-sp/hard/libc_nano.a(lib_a-abort.o)
 .debug_frame   0x0000000000000cc0       0x28 /opt/ti/ccsv7/tools/compiler/gcc-arm-none-eabi-6-2017-q1-update/bin/../lib/gcc/arm-none-eabi/6.3.1/../../../../arm-none-eabi/lib/thumb/v7e-m/fpv4-sp/hard/libc_nano.a(lib_a-cxa_atexit.o)
 .debug_frame   0x0000000000000ce8       0x30 /opt/ti/ccsv7/tools/compiler/gcc-arm-none-eabi-6-2017-q1-update/bin/../lib/gcc/arm-none-eabi/6.3.1/../../../../arm-none-eabi/lib/thumb/v7e-m/fpv4-sp/hard/libc_nano.a(lib_a-malloc.o)
 .debug_frame   0x0000000000000d18       0x38 /opt/ti/ccsv7/tools/compiler/gcc-arm-none-eabi-6-2017-q1-update/bin/../lib/gcc/arm-none-eabi/6.3.1/../../../../arm-none-eabi/lib/thumb/v7e-m/fpv4-sp/hard/libc_nano.a(lib_a-nano-freer.o)
 .debug_frame   0x0000000000000d50       0x2c /opt/ti/ccsv7/tools/compiler/gcc-arm-none-eabi-6-2017-q1-update/bin/../lib/gcc/arm-none-eabi/6.3.1/../../../../arm-none-eabi/lib/thumb/v7e-m/fpv4-sp/hard/libc_nano.a(lib_a-nano-mallocr.o)
 .debug_frame   0x0000000000000d7c       0x2c /opt/ti/ccsv7/tools/compiler/gcc-arm-none-eabi-6-2017-q1-update/bin/../lib/gcc/arm-none-eabi/6.3.1/../../../../arm-none-eabi/lib/thumb/v7e-m/fpv4-sp/hard/libc_nano.a(lib_a-sbrkr.o)
 .debug_frame   0x0000000000000da8       0xcc /opt/ti/ccsv7/tools/compiler/gcc-arm-none-eabi-6-2017-q1-update/bin/../lib/gcc/arm-none-eabi/6.3.1/../../../../arm-none-eabi/lib/thumb/v7e-m/fpv4-sp/hard/libc_nano.a(lib_a-signal.o)
 .debug_frame   0x0000000000000e74       0x3c /opt/ti/ccsv7/tools/compiler/gcc-arm-none-eabi-6-2017-q1-update/bin/../lib/gcc/arm-none-eabi/6.3.1/../../../../arm-none-eabi/lib/thumb/v7e-m/fpv4-sp/hard/libc_nano.a(lib_a-signalr.o)
 .debug_frame   0x0000000000000eb0       0x20 /opt/ti/ccsv7/tools/compiler/gcc-arm-none-eabi-6-2017-q1-update/bin/../lib/gcc/arm-none-eabi/6.3.1/../../../../arm-none-eabi/lib/thumb/v7e-m/fpv4-sp/hard/libc_nano.a(lib_a-strcmp.o)
 .debug_frame   0x0000000000000ed0       0x30 /opt/ti/ccsv7/tools/compiler/gcc-arm-none-eabi-6-2017-q1-update/bin/../lib/gcc/arm-none-eabi/6.3.1/../../../../arm-none-eabi/lib/thumb/v7e-m/fpv4-sp/hard/libc_nano.a(lib_a-mlock.o)
 .debug_frame   0x0000000000000f00       0x5c /opt/ti/ccsv7/tools/compiler/gcc-arm-none-eabi-6-2017-q1-update/bin/../lib/gcc/arm-none-eabi/6.3.1/../../../../arm-none-eabi/lib/thumb/v7e-m/fpv4-sp/hard/libc_nano.a(lib_a-reent.o)
 .debug_frame   0x0000000000000f5c       0x20 /opt/ti/ccsv7/tools/compiler/gcc-arm-none-eabi-6-2017-q1-update/bin/../lib/gcc/arm-none-eabi/6.3.1/../../../../arm-none-eabi/lib/thumb/v7e-m/fpv4-sp/hard/libnosys.a(getpid.o)
 .debug_frame   0x0000000000000f7c       0x20 /opt/ti/ccsv7/tools/compiler/gcc-arm-none-eabi-6-2017-q1-update/bin/../lib/gcc/arm-none-eabi/6.3.1/../../../../arm-none-eabi/lib/thumb/v7e-m/fpv4-sp/hard/libnosys.a(kill.o)
 .debug_frame   0x0000000000000f9c       0x20 /opt/ti/ccsv7/tools/compiler/gcc-arm-none-eabi-6-2017-q1-update/bin/../lib/gcc/arm-none-eabi/6.3.1/../../../../arm-none-eabi/lib/thumb/v7e-m/fpv4-sp/hard/libnosys.a(sbrk.o)

.debug_info     0x0000000000000000     0x37e6
 .debug_info    0x0000000000000000      0x992 Debug/main.cpp.o
 .debug_info    0x0000000000000992      0x149 Debug/startup_msp432p401r_gcc.c.o
 .debug_info    0x0000000000000adb      0xd1b Debug/system_msp432p401r.c.o
 .debug_info    0x00000000000017f6     0x13b1 /home/student/git/workspace_mct/YAHAL/libYAHAL_msp432.a(gpio_msp432.cpp.o)
 .debug_info    0x0000000000002ba7      0xc3f /home/student/git/workspace_mct/YAHAL/libYAHAL_msp432.a(timer_msp432.cpp.o)

.debug_abbrev   0x0000000000000000      0xc6f
 .debug_abbrev  0x0000000000000000      0x32a Debug/main.cpp.o
 .debug_abbrev  0x000000000000032a       0xbd Debug/startup_msp432p401r_gcc.c.o
 .debug_abbrev  0x00000000000003e7      0x115 Debug/system_msp432p401r.c.o
 .debug_abbrev  0x00000000000004fc      0x3ef /home/student/git/workspace_mct/YAHAL/libYAHAL_msp432.a(gpio_msp432.cpp.o)
 .debug_abbrev  0x00000000000008eb      0x384 /home/student/git/workspace_mct/YAHAL/libYAHAL_msp432.a(timer_msp432.cpp.o)

.debug_aranges  0x0000000000000000      0x248
 .debug_aranges
                0x0000000000000000       0x60 Debug/main.cpp.o
 .debug_aranges
                0x0000000000000060       0x28 Debug/startup_msp432p401r_gcc.c.o
 .debug_aranges
                0x0000000000000088       0x28 Debug/system_msp432p401r.c.o
 .debug_aranges
                0x00000000000000b0       0xf0 /home/student/git/workspace_mct/YAHAL/libYAHAL_msp432.a(gpio_msp432.cpp.o)
 .debug_aranges
                0x00000000000001a0       0xa8 /home/student/git/workspace_mct/YAHAL/libYAHAL_msp432.a(timer_msp432.cpp.o)

.debug_ranges   0x0000000000000000      0x1f8
 .debug_ranges  0x0000000000000000       0x50 Debug/main.cpp.o
 .debug_ranges  0x0000000000000050       0x18 Debug/startup_msp432p401r_gcc.c.o
 .debug_ranges  0x0000000000000068       0x18 Debug/system_msp432p401r.c.o
 .debug_ranges  0x0000000000000080       0xe0 /home/student/git/workspace_mct/YAHAL/libYAHAL_msp432.a(gpio_msp432.cpp.o)
 .debug_ranges  0x0000000000000160       0x98 /home/student/git/workspace_mct/YAHAL/libYAHAL_msp432.a(timer_msp432.cpp.o)

.debug_line     0x0000000000000000      0xec6
 .debug_line    0x0000000000000000      0x32f Debug/main.cpp.o
 .debug_line    0x000000000000032f      0x13b Debug/startup_msp432p401r_gcc.c.o
 .debug_line    0x000000000000046a      0x259 Debug/system_msp432p401r.c.o
 .debug_line    0x00000000000006c3      0x4aa /home/student/git/workspace_mct/YAHAL/libYAHAL_msp432.a(gpio_msp432.cpp.o)
 .debug_line    0x0000000000000b6d      0x359 /home/student/git/workspace_mct/YAHAL/libYAHAL_msp432.a(timer_msp432.cpp.o)

.debug_str      0x0000000000000000     0x1e19
 .debug_str     0x0000000000000000      0x7b4 Debug/main.cpp.o
                                        0x858 (size before relaxing)
 .debug_str     0x00000000000007b4      0x1aa Debug/startup_msp432p401r_gcc.c.o
                                        0x288 (size before relaxing)
 .debug_str     0x000000000000095e      0x8b4 Debug/system_msp432p401r.c.o
                                        0xb1b (size before relaxing)
 .debug_str     0x0000000000001212      0x712 /home/student/git/workspace_mct/YAHAL/libYAHAL_msp432.a(gpio_msp432.cpp.o)
                                        0xd18 (size before relaxing)
 .debug_str     0x0000000000001924      0x4f5 /home/student/git/workspace_mct/YAHAL/libYAHAL_msp432.a(timer_msp432.cpp.o)
                                        0xb40 (size before relaxing)

.stab           0x0000000000000000       0x3c
 .stab          0x0000000000000000       0x24 /opt/ti/ccsv7/tools/compiler/gcc-arm-none-eabi-6-2017-q1-update/bin/../lib/gcc/arm-none-eabi/6.3.1/../../../../arm-none-eabi/lib/thumb/v7e-m/fpv4-sp/hard/libnosys.a(getpid.o)
 .stab          0x0000000000000024       0x18 /opt/ti/ccsv7/tools/compiler/gcc-arm-none-eabi-6-2017-q1-update/bin/../lib/gcc/arm-none-eabi/6.3.1/../../../../arm-none-eabi/lib/thumb/v7e-m/fpv4-sp/hard/libnosys.a(kill.o)
                                         0x24 (size before relaxing)

.stabstr        0x0000000000000000       0x76
 .stabstr       0x0000000000000000       0x76 /opt/ti/ccsv7/tools/compiler/gcc-arm-none-eabi-6-2017-q1-update/bin/../lib/gcc/arm-none-eabi/6.3.1/../../../../arm-none-eabi/lib/thumb/v7e-m/fpv4-sp/hard/libnosys.a(getpid.o)
